 sim

 Timestamp is 4fb05c7d (Mon May 14 13:14:37 2012)

 Preferred load address is 10000000

 Start         Length     Name                   Class
 0001:00000000 00004198H .rdata                  CODE
 0001:00004198 00000020H .rdata$debug            CODE
 0001:000041b8 0000e178H .text                   CODE
 0001:00012330 00000040H .xdata                  CODE
 0001:00012370 0000003cH .idata$2                CODE
 0001:000123ac 00000014H .idata$3                CODE
 0001:000123c0 000000e8H .idata$4                CODE
 0001:000124a8 000000a2H .idata$6                CODE
 0001:00012550 000000ffH .edata                  CODE
 0002:00000000 000000e8H .idata$5                DATA
 0002:000000e8 000007d8H .data                   DATA
 0002:000008c0 0000004cH .bss                    DATA
 0003:00000000 000002b0H .pdata                  DATA

  Address         Publics by Value              Rva+Base       Lib:Object

 0000:00000000       ___safe_se_handler_count   00000000     <absolute>
 0000:00000000       ___safe_se_handler_table   00000000     <absolute>
 0001:000000b0       ??_C@_1CK@BGADNIHC@?$AAD?$AAL?$AAL?$AA_?$AAP?$AAR?$AAO?$AAC?$AAE?$AAS?$AAS?$AA_?$AAD?$AAE?$AAT?$AAA?$AAC?$AAH?$AA?$AN?$AA?6?$AA?$AA@ 100010b0     sim_common_topaz_v1:simce.obj
 0001:000000dc       ??_C@_1CK@LKLGBGJK@?$AAD?$AAL?$AAL?$AA_?$AAP?$AAR?$AAO?$AAC?$AAE?$AAS?$AAS?$AA_?$AAA?$AAT?$AAT?$AAA?$AAC?$AAH?$AA?$AN?$AA?6?$AA?$AA@ 100010dc     sim_common_topaz_v1:simce.obj
 0001:00000108       ??_C@_1BG@GLDHNJAK@?$AA?9?$AAS?$AAC?$AAR?$AA_?$AAI?$AAn?$AAi?$AAt?$AA?6?$AA?$AA@ 10001108     sim_common_topaz_v1:simce.obj
 0001:00000120       ??_C@_1FK@FNONLNGN@?$AA?$CF?$AAs?$AA?3?$AA?5?$AAD?$AAE?$AAB?$AAU?$AAG?$AAC?$AAH?$AAK?$AA?5?$AAf?$AAa?$AAi?$AAl?$AAe?$AAd?$AA?5?$AAi?$AAn?$AA?5?$AAf?$AAi?$AAl?$AAe?$AA?5?$AA?$CF?$AAs?$AA?5?$AAa@ 10001120     sim_common_topaz_v1:simce.obj
 0001:0000017c       ??_C@_1BA@LEPJIIOK@?$AAU?$AAn?$AAk?$AAn?$AAo?$AAw?$AAn?$AA?$AA@ 1000117c     sim_common_topaz_v1:simce.obj
 0001:00000190       ??_C@_1KG@IHHDNDD@?$AAC?$AA?3?$AA?2?$AAW?$AAI?$AAN?$AAC?$AAE?$AAR?$AAO?$AAO?$AAT?$AAS?$AA?2?$AAT?$AAo?$AAp?$AAa?$AAz?$AA?2?$AAW?$AAI?$AAN?$AAC?$AAE?$AA6?$AA0?$AA0?$AA?2?$AAP?$AAL?$AAA@ 10001190     sim_common_topaz_v1:simce.obj
 0001:00000238       ??_C@_1EC@JOJIADHI@?$AAS?$AAC?$AAR?$AA_?$AAI?$AAn?$AAi?$AAt?$AA?5?$AAD?$AAe?$AAv?$AAi?$AAc?$AAe?$AA?5?$AAO?$AAv?$AAe?$AAr?$AAf?$AAl?$AAo?$AAw?$AA?5?$AAe?$AAr?$AAr?$AAo?$AAr?$AA?$AN?$AA?6@ 10001238     sim_common_topaz_v1:simce.obj
 0001:0000027c       ??_C@_1BG@BJMGIDIK@?$AA?$CL?$AAS?$AAC?$AAR?$AA_?$AAI?$AAn?$AAi?$AAt?$AA?6?$AA?$AA@ 1000127c     sim_common_topaz_v1:simce.obj
 0001:00000294       ??_C@_1BM@ICLGOIPP@?$AA?9?$AAS?$AAC?$AAR?$AA_?$AAD?$AAe?$AAi?$AAn?$AAi?$AAt?$AA?$AN?$AA?6?$AA?$AA@ 10001294     sim_common_topaz_v1:simce.obj
 0001:000002b0       ??_C@_1BM@IHAKOGLB@?$AA?$CL?$AAS?$AAC?$AAR?$AA_?$AAD?$AAe?$AAi?$AAn?$AAi?$AAt?$AA?$AN?$AA?6?$AA?$AA@ 100012b0     sim_common_topaz_v1:simce.obj
 0001:000002cc       ??_C@_1BG@EIIPPJAD@?$AA?9?$AAS?$AAC?$AAR?$AA_?$AAO?$AAp?$AAe?$AAn?$AA?6?$AA?$AA@ 100012cc     sim_common_topaz_v1:simce.obj
 0001:000002e4       ??_C@_1BM@LCEJNAKA@?$AAC?$AAa?$AAr?$AAd?$AAS?$AAt?$AAa?$AAt?$AAe?$AA?5?$AA?$CF?$AAd?$AA?6?$AA?$AA@ 100012e4     sim_common_topaz_v1:simce.obj
 0001:00000300       ??_C@_1DC@MMHDNFIG@?$AAO?$AAp?$AAe?$AAn?$AA?5?$AA?9?$AA?5?$AAi?$AAn?$AAv?$AAa?$AAl?$AAi?$AAd?$AA?5?$AAs?$AAt?$AAa?$AAt?$AAe?$AA?5?$AA?$CF?$AAd?$AA?6?$AA?$AA@ 10001300     sim_common_topaz_v1:simce.obj
 0001:00000334       ??_C@_1BO@BMJLDEBA@?$AA?$CL?$AAS?$AAC?$AAR?$AA_?$AAO?$AAp?$AAe?$AAn?$AA?$CI?$AA?$CF?$AAx?$AA?$CJ?$AA?6?$AA?$AA@ 10001334     sim_common_topaz_v1:simce.obj
 0001:00000358       ??_C@_1EI@KPFPBOEF@?$AAV?$AAa?$AAl?$AAi?$AAd?$AAa?$AAt?$AAe?$AAD?$AAe?$AAv?$AAi?$AAc?$AAe?$AA?5?$AA?9?$AA?5?$AAI?$AAn?$AAv?$AAa?$AAl?$AAi?$AAd?$AA?5?$AAO?$AAb?$AAj?$AAe?$AAc?$AAt?$AA?5@ 10001358     sim_common_topaz_v1:simce.obj
 0001:000003a0       ??_C@_1GE@BCEANOJG@?$AA?9?$AAS?$AAI?$AAM?$AAC?$AAa?$AAr?$AAd?$AAD?$AAe?$AAt?$AAe?$AAc?$AAt?$AAi?$AAo?$AAn?$AAT?$AAh?$AAr?$AAe?$AAa?$AAd?$AA?5?$AAT?$AAe?$AAr?$AAm?$AAi?$AAn?$AAa?$AAt@ 100013a0     sim_common_topaz_v1:simce.obj
 0001:00000408       ??_C@_1EE@GCLLBLKJ@?$AAS?$AAI?$AAM?$AAC?$AAa?$AAr?$AAd?$AAD?$AAe?$AAt?$AAe?$AAc?$AAt?$AAi?$AAo?$AAn?$AAT?$AAh?$AAr?$AAe?$AAa?$AAd?$AA?5?$AA?9?$AA?5?$AAC?$AAa?$AAr?$AAd?$AA?5?$AA?$CF?$AAs@ 10001408     sim_common_topaz_v1:simce.obj
 0001:0000044c       ??_C@_1BC@IOMLCCNH@?$AAi?$AAn?$AAs?$AAe?$AAr?$AAt?$AAe?$AAd?$AA?$AA@ 1000144c     sim_common_topaz_v1:simce.obj
 0001:00000460       ??_C@_1BA@FDKPJHCF@?$AAr?$AAe?$AAm?$AAo?$AAv?$AAe?$AAd?$AA?$AA@ 10001460     sim_common_topaz_v1:simce.obj
 0001:00000470       ??_C@_1GC@JIIEBLHH@?$AA?$CL?$AAS?$AAI?$AAM?$AAC?$AAa?$AAr?$AAd?$AAD?$AAe?$AAt?$AAe?$AAc?$AAt?$AAi?$AAo?$AAn?$AAT?$AAh?$AAr?$AAe?$AAa?$AAd?$AA?5?$AAE?$AAn?$AAt?$AAe?$AAr?$AAi?$AAn?$AAg@ 10001470     sim_common_topaz_v1:simce.obj
 0001:000004d4       ??_C@_1BI@BKBFNLCM@?$AA?$CL?$AAS?$AAC?$AAR?$AA_?$AAC?$AAl?$AAo?$AAs?$AAe?$AA?6?$AA?$AA@ 100014d4     sim_common_topaz_v1:simce.obj
 0001:000004f0       ??_C@_1FA@NJGJJLKL@?$AAC?$AAl?$AAo?$AAs?$AAe?$AA?5?$AA?9?$AA?5?$AAw?$AAa?$AAi?$AAt?$AAi?$AAn?$AAg?$AA?5?$AAf?$AAo?$AAr?$AA?5?$AA?$CF?$AAd?$AA?5?$AAt?$AAh?$AAr?$AAe?$AAa?$AAd?$AAs?$AA?5?$AAt@ 100014f0     sim_common_topaz_v1:simce.obj
 0001:00000540       ??_C@_1DE@KCNMICLP@?$AA?$CL?$AAS?$AAC?$AAR?$AA_?$AAC?$AAl?$AAo?$AAs?$AAe?$AA?$CI?$AA?$CF?$AAx?$AA?$CJ?$AA?5?$AA?9?$AA?5?$AAe?$AAn?$AAt?$AAe?$AAr?$AAe?$AAd?$AA?6?$AA?$AA@ 10001540     sim_common_topaz_v1:simce.obj
 0001:00000574       ??_C@_1CA@HMFKFEEP@?$AA?9?$AAS?$AAC?$AAR?$AA_?$AAI?$AAO?$AAC?$AAo?$AAn?$AAt?$AAr?$AAo?$AAl?$AA?6?$AA?$AA@ 10001574     sim_common_topaz_v1:simce.obj
 0001:00000598       ??_C@_1EA@HOJDOEIN@?$AAD?$AAe?$AAv?$AAi?$AAc?$AAe?$AAI?$AAO?$AAC?$AAT?$AAL?$AA?5?$AA?9?$AA?5?$AAi?$AAn?$AAv?$AAa?$AAl?$AAi?$AAd?$AA?5?$AAs?$AAt?$AAa?$AAt?$AAe?$AA?5?$AA?$CF?$AAd?$AA?6?$AA?$AA@ 10001598     sim_common_topaz_v1:simce.obj
 0001:000005d8       ??_C@_1CA@DFBFEDHA@?$AA?$CL?$AAS?$AAC?$AAR?$AA_?$AAI?$AAO?$AAC?$AAo?$AAn?$AAt?$AAr?$AAo?$AAl?$AA?6?$AA?$AA@ 100015d8     sim_common_topaz_v1:simce.obj
 0001:000005f8       ??_C@_1CK@DLNMCBLB@?$AAP?$AAo?$AAw?$AAe?$AAr?$AAU?$AAp?$AA?$CI?$AA?$CJ?$AA?5?$AA?9?$AA?5?$AAe?$AAn?$AAt?$AAe?$AAr?$AAe?$AAd?$AA?6?$AA?$AA@ 100015f8     sim_common_topaz_v1:simce.obj
 0001:00000624       ??_C@_1CO@LIPKJBJ@?$AAP?$AAo?$AAw?$AAe?$AAr?$AAD?$AAo?$AAw?$AAn?$AA?$CI?$AA?$CJ?$AA?5?$AA?9?$AA?5?$AAe?$AAn?$AAt?$AAe?$AAr?$AAe?$AAd?$AA?6?$AA?$AA@ 10001624     sim_common_topaz_v1:simce.obj
 0001:00000654       ??_C@_1CA@HGFIDHDL@?$AA?9?$AAS?$AAI?$AAM?$AAL?$AAo?$AAa?$AAd?$AAD?$AAe?$AAv?$AAi?$AAc?$AAe?$AA?6?$AA?$AA@ 10001654     sim_common_topaz_v1:simce.obj
 0001:00000674       ??_C@_1DE@CBDBAGOJ@?$AAS?$AAI?$AAM?$AAC?$AAr?$AAe?$AAa?$AAt?$AAe?$AAD?$AAe?$AAv?$AAi?$AAc?$AAe?$AA?3?$AA?5?$AAE?$AAx?$AAi?$AAt?$AA?5?$AA?$CF?$AAx?$AA?6?$AA?$AA@ 10001674     sim_common_topaz_v1:simce.obj
 0001:000006a8       ??_C@_1EC@PHEFAHEO@?$AAS?$AAm?$AAa?$AAr?$AAt?$AAc?$AAa?$AAr?$AAd?$AAI?$AAn?$AAi?$AAt?$AAi?$AAa?$AAl?$AAi?$AAz?$AAe?$AA?5?$AAf?$AAa?$AAi?$AAl?$AAe?$AAd?$AA?5?$AA?9?$AA?5?$AA?$CF?$AAx?$AA?6@ 100016a8     sim_common_topaz_v1:simce.obj
 0001:000006ec       ??_C@_03JAFGGFOK@Sim?$AA@  100016ec     sim_common_topaz_v1:simce.obj
 0001:000006f0       ??_C@_09JJPIIJJC@Freescale?$AA@ 100016f0     sim_common_topaz_v1:simce.obj
 0001:000006fc       ??_C@_1CA@DPBHCAAE@?$AA?$CL?$AAS?$AAI?$AAM?$AAL?$AAo?$AAa?$AAd?$AAD?$AAe?$AAv?$AAi?$AAc?$AAe?$AA?6?$AA?$AA@ 100016fc     sim_common_topaz_v1:simce.obj
 0001:0000071c       ??_C@_1CO@JFJEPDDF@?$AA?9?$AAS?$AAI?$AAM?$AAV?$AAe?$AAn?$AAd?$AAo?$AAr?$AAI?$AAo?$AAc?$AAt?$AAl?$AA?5?$AA?$CI?$AA?$CF?$AAl?$AAx?$AA?$CJ?$AA?6?$AA?$AA@ 1000171c     sim_common_topaz_v1:simce.obj
 0001:0000074c       ??_C@_1CC@MKKOGKAA@?$AA?$CL?$AAS?$AAI?$AAM?$AAV?$AAe?$AAn?$AAd?$AAo?$AAr?$AAI?$AAo?$AAc?$AAt?$AAl?$AA?6?$AA?$AA@ 1000174c     sim_common_topaz_v1:simce.obj
 0001:00000770       ??_C@_19OBNDINH@?$AAP?$AAo?$AAr?$AAt?$AA?$AA@ 10001770     sim_common_topaz_v1:simce.obj
 0001:00000780       ??_C@_1FO@DFGLELPC@?$AAG?$AAe?$AAt?$AAI?$AAO?$AAI?$AAn?$AAd?$AAe?$AAx?$AA?5?$AA?9?$AA?5?$AAR?$AAe?$AAg?$AAQ?$AAu?$AAe?$AAr?$AAy?$AAV?$AAa?$AAl?$AAu?$AAe?$AAE?$AAx?$AA?$CI?$AA?$CF?$AAs?$AA?$CJ@ 10001780     sim_common_topaz_v1:simce.obj
 0001:000007e0       ??_C@_1CC@KMPFMANC@?$AAD?$AAe?$AAv?$AAi?$AAc?$AAe?$AAA?$AAr?$AAr?$AAa?$AAy?$AAI?$AAn?$AAd?$AAe?$AAx?$AA?$AA@ 100017e0     sim_common_topaz_v1:simce.obj
 0001:00000808       ??_C@_1FE@PBAJMNGE@?$AAG?$AAe?$AAt?$AAI?$AAO?$AAI?$AAn?$AAd?$AAe?$AAx?$AA?5?$AAO?$AAp?$AAe?$AAn?$AAD?$AAe?$AAv?$AAi?$AAc?$AAe?$AAK?$AAe?$AAy?$AA?5?$AAr?$AAe?$AAt?$AAu?$AAr?$AAn?$AAe@ 10001808     sim_common_topaz_v1:simce.obj
 0001:00000860       ??_C@_1GE@DPLNBFDK@?$AAG?$AAe?$AAt?$AAD?$AAe?$AAv?$AAi?$AAc?$AAe?$AAN?$AAa?$AAm?$AAe?$AA?5?$AA?9?$AA?5?$AAR?$AAe?$AAg?$AAQ?$AAu?$AAe?$AAr?$AAy?$AAV?$AAa?$AAl?$AAu?$AAe?$AAE?$AAx?$AA?$CI@ 10001860     sim_common_topaz_v1:simce.obj
 0001:000008c4       ??_C@_19DINFBLAK@?$AAN?$AAa?$AAm?$AAe?$AA?$AA@ 100018c4     sim_common_topaz_v1:simce.obj
 0001:000008d0       ??_C@_1GI@HCFPLBGJ@?$AAG?$AAe?$AAt?$AAD?$AAe?$AAv?$AAi?$AAc?$AAe?$AAN?$AAa?$AAm?$AAe?$AA?5?$AAR?$AAe?$AAg?$AAO?$AAp?$AAe?$AAn?$AAK?$AAe?$AAy?$AAE?$AAx?$AA?$CI?$AAH?$AAL?$AAM?$AA?2?$AA?$CF@ 100018d0     sim_common_topaz_v1:simce.obj
 0001:00000938       ??_C@_19GFKPKJIA@?$AA?5?$AA?$FL?$AA?5?$AA?$FN?$AA?$AA@ 10001938     sim_common_topaz_v1:simce.obj
 0001:00000944       ??_C@_1CE@HDIJNJPD@?$AA?9?$AAS?$AAI?$AAM?$AAU?$AAn?$AAl?$AAo?$AAa?$AAd?$AAD?$AAe?$AAv?$AAi?$AAc?$AAe?$AA?6?$AA?$AA@ 10001944     sim_common_topaz_v1:simce.obj
 0001:00000968       ??_C@_1EM@GKBAGMBK@?$AA?$CF?$AAs?$AA?3?$AAU?$AAn?$AAl?$AAo?$AAa?$AAd?$AAD?$AAe?$AAv?$AAi?$AAc?$AAe?$AA?5?$AA?9?$AA?5?$AAf?$AAr?$AAe?$AAe?$AAi?$AAn?$AAg?$AA?5?$AAr?$AAe?$AAs?$AAo?$AAu?$AAr@ 10001968     sim_common_topaz_v1:simce.obj
 0001:000009b8       ??_C@_1HC@LCFDEFPP@?$AAU?$AAn?$AAl?$AAo?$AAa?$AAd?$AAD?$AAe?$AAv?$AAi?$AAc?$AAe?$AA?5?$AA?9?$AA?5?$AAw?$AAa?$AAi?$AAt?$AAi?$AAn?$AAg?$AA?5?$AAf?$AAo?$AAr?$AA?5?$AAr?$AAe?$AAf?$AAC?$AAo@ 100019b8     sim_common_topaz_v1:simce.obj
 0001:00000a2c       ??_C@_1CE@LKEJCOAP@?$AA?$CL?$AAS?$AAI?$AAM?$AAU?$AAn?$AAl?$AAo?$AAa?$AAd?$AAD?$AAe?$AAv?$AAi?$AAc?$AAe?$AA?6?$AA?$AA@ 10001a2c     sim_common_topaz_v1:simce.obj
 0001:00000a50       ??_C@_1BE@NGBNOKJN@?$AAW?$AAa?$AAr?$AAm?$AAR?$AAe?$AAs?$AAe?$AAt?$AA?$AA@ 10001a50     sim_common_topaz_v1:simcb.obj
 0001:00000a64       ??_C@_1BE@JOIIPBN@?$AAC?$AAo?$AAl?$AAd?$AAR?$AAe?$AAs?$AAe?$AAt?$AA?$AA@ 10001a64     sim_common_topaz_v1:simcb.obj
 0001:00000a78       ??_C@_1BE@IFHEBOLO@?$AAP?$AAo?$AAw?$AAe?$AAr?$AAD?$AAo?$AAw?$AAn?$AA?$AA@ 10001a78     sim_common_topaz_v1:simcb.obj
 0001:00000a8c       ??_C@_1CO@PLKEHLGK@?$AA?9?$AAC?$AAB?$AAC?$AAa?$AAr?$AAd?$AAP?$AAo?$AAw?$AAe?$AAr?$AA?5?$AAE?$AAx?$AAi?$AAt?$AA?3?$AA?5?$AA?$CF?$AAX?$AA?6?$AA?$AA@ 10001a8c     sim_common_topaz_v1:simcb.obj
 0001:00000abc       ??_C@_1DI@BDEOAOOD@?$AA?$CL?$AAC?$AAB?$AAC?$AAa?$AAr?$AAd?$AAP?$AAo?$AAw?$AAe?$AAr?$AA?0?$AA?5?$AAR?$AAe?$AAq?$AAu?$AAe?$AAs?$AAt?$AA?5?$AA?$DN?$AA?5?$AA?$CF?$AAs?$AA?6?$AA?$AA@ 10001abc     sim_common_topaz_v1:simcb.obj
 0001:00000af4       ??_C@_1DC@EAHEDIHO@?$AA?9?$AAC?$AAB?$AAS?$AAe?$AAt?$AAP?$AAr?$AAo?$AAt?$AAo?$AAc?$AAo?$AAl?$AA?3?$AA?5?$AAE?$AAx?$AAi?$AAt?$AA?5?$AA?$CF?$AAX?$AA?6?$AA?$AA@ 10001af4     sim_common_topaz_v1:simcb.obj
 0001:00000b28       ??_C@_1CM@ECJKAPBF@?$AA?$CL?$AAC?$AAB?$AAS?$AAe?$AAt?$AAP?$AAr?$AAo?$AAt?$AAo?$AAc?$AAo?$AAl?$AA?5?$AAE?$AAn?$AAt?$AAe?$AAr?$AA?6?$AA?$AA@ 10001b28     sim_common_topaz_v1:simcb.obj
 0001:00000b54       ??_C@_1CM@KNOPAAPP@?$AA?9?$AAC?$AAB?$AAT?$AAr?$AAa?$AAn?$AAs?$AAm?$AAi?$AAt?$AA?5?$AAE?$AAx?$AAi?$AAt?$AA?3?$AA?5?$AA?$CF?$AAX?$AA?6?$AA?$AA@ 10001b54     sim_common_topaz_v1:simcb.obj
 0001:00000b80       ??_C@_1FO@FFEMGIOI@?$AAR?$AAA?$AAW?$AA?5?$AAp?$AAr?$AAo?$AAt?$AAo?$AAc?$AAo?$AAl?$AA?5?$AAi?$AAs?$AA?5?$AAn?$AAo?$AAt?$AA?5?$AAs?$AAu?$AAp?$AAp?$AAo?$AAr?$AAt?$AAe?$AAd?$AA?5?$AAi?$AAn@ 10001b80     sim_common_topaz_v1:simcb.obj
 0001:00000be0       ??_C@_1FM@PCHCLDGC@?$AAT?$AA1?$AA?5?$AAp?$AAr?$AAo?$AAt?$AAo?$AAc?$AAo?$AAl?$AA?5?$AAi?$AAs?$AA?5?$AAn?$AAo?$AAt?$AA?5?$AAs?$AAu?$AAp?$AAp?$AAo?$AAr?$AAt?$AAe?$AAd?$AA?5?$AAi?$AAn?$AA?5@ 10001be0     sim_common_topaz_v1:simcb.obj
 0001:00000c3c       ??_C@_1CG@DBOLLHEN@?$AA?$CL?$AAC?$AAB?$AAT?$AAr?$AAa?$AAn?$AAs?$AAm?$AAi?$AAt?$AA?5?$AAE?$AAn?$AAt?$AAe?$AAr?$AA?6?$AA?$AA@ 10001c3c     sim_common_topaz_v1:simcb.obj
 0001:00000c64       ??_C@_1DA@CFDDNKDP@?$AA?9?$AAC?$AAB?$AAT?$AA0?$AAT?$AAr?$AAa?$AAn?$AAs?$AAm?$AAi?$AAt?$AA?5?$AAE?$AAx?$AAi?$AAt?$AA?3?$AA?5?$AA?$CF?$AAX?$AA?6?$AA?$AA@ 10001c64     sim_common_topaz_v1:simcb.obj
 0001:00000c94       ??_C@_1CK@CICBFFEH@?$AA?$CL?$AAC?$AAB?$AAT?$AA0?$AAT?$AAr?$AAa?$AAn?$AAs?$AAm?$AAi?$AAt?$AA?5?$AAE?$AAn?$AAt?$AAe?$AAr?$AA?6?$AA?$AA@ 10001c94     sim_common_topaz_v1:simcb.obj
 0001:00000cc0       ??_C@_1DA@CFNGPMKN@?$AA?9?$AAT?$AA0?$AA_?$AAE?$AAx?$AAc?$AAh?$AAa?$AAn?$AAg?$AAe?$AAD?$AAa?$AAt?$AAa?$AA?5?$AAE?$AAn?$AAt?$AAe?$AAr?$AA?6?$AA?$AA@ 10001cc0     sim_common_topaz_v1:simcb.obj
 0001:00000cf0       ??_C@_1DA@KIHCJGGF@?$AA?$CL?$AAT?$AA0?$AA_?$AAE?$AAx?$AAc?$AAh?$AAa?$AAn?$AAg?$AAe?$AAD?$AAa?$AAt?$AAa?$AA?5?$AAE?$AAn?$AAt?$AAe?$AAr?$AA?6?$AA?$AA@ 10001cf0     sim_common_topaz_v1:simcb.obj
 0001:00000d20       ??_C@_1CC@DIAMDOKD@?$AA?9?$AAC?$AAB?$AAC?$AAa?$AAr?$AAd?$AAT?$AAr?$AAa?$AAc?$AAk?$AAi?$AAn?$AAg?$AA?6?$AA?$AA@ 10001d20     sim_common_topaz_v1:simcb.obj
 0001:00000d44       ??_C@_1CC@ODABNIBH@?$AA?$CL?$AAC?$AAB?$AAC?$AAa?$AAr?$AAd?$AAT?$AAr?$AAa?$AAc?$AAk?$AAi?$AAn?$AAg?$AA?6?$AA?$AA@ 10001d44     sim_common_topaz_v1:simcb.obj
 0001:00000d68       ??_C@_1CG@EOMOFCAJ@?$AA?9?$AAC?$AAB?$AAS?$AAy?$AAn?$AAc?$AAh?$AAr?$AAo?$AAn?$AAi?$AAz?$AAe?$AAS?$AAI?$AAM?$AA?6?$AA?$AA@ 10001d68     sim_common_topaz_v1:simcb.obj
 0001:00000d90       ??_C@_1EA@EBHONLAA@?$AAP?$AAr?$AAo?$AAb?$AAl?$AAe?$AAm?$AAs?$AA?5?$AAi?$AAn?$AA?5?$AAt?$AAi?$AAm?$AAe?$AA?5?$AAc?$AAo?$AAn?$AAf?$AAi?$AAg?$AAu?$AAr?$AAa?$AAt?$AAi?$AAo?$AAn?$AA?6?$AA?$AA@ 10001d90     sim_common_topaz_v1:simcb.obj
 0001:00000dd0       ??_C@_1EC@OBJGMIBD@?$AAP?$AAr?$AAo?$AAb?$AAl?$AAe?$AAm?$AAs?$AA?5?$AAi?$AAn?$AA?5?$AAc?$AAl?$AAo?$AAc?$AAk?$AA?5?$AAc?$AAo?$AAn?$AAf?$AAi?$AAg?$AAu?$AAr?$AAa?$AAt?$AAi?$AAo?$AAn?$AA?6@ 10001dd0     sim_common_topaz_v1:simcb.obj
 0001:00000e14       ??_C@_1CG@NFBOFCMH@?$AA?$CL?$AAC?$AAB?$AAS?$AAy?$AAn?$AAc?$AAh?$AAr?$AAo?$AAn?$AAi?$AAz?$AAe?$AAS?$AAI?$AAM?$AA?6?$AA?$AA@ 10001e14     sim_common_topaz_v1:simcb.obj
 0001:00000e3c       ??_C@_1CI@COLNEDCD@?$AA?9?$AAC?$AAB?$AAU?$AAp?$AAd?$AAa?$AAt?$AAe?$AAC?$AAa?$AAr?$AAd?$AAS?$AAt?$AAa?$AAt?$AAe?$AA?6?$AA?$AA@ 10001e3c     sim_common_topaz_v1:simcb.obj
 0001:00000e64       ??_C@_1CI@HLMECCDD@?$AA?$CL?$AAC?$AAB?$AAU?$AAp?$AAd?$AAa?$AAt?$AAe?$AAC?$AAa?$AAr?$AAd?$AAS?$AAt?$AAa?$AAt?$AAe?$AA?6?$AA?$AA@ 10001e64     sim_common_topaz_v1:simcb.obj
 0001:00000f10       ??_C@_1EG@OOODBOJK@?$AA?9?$AAS?$AAI?$AAM?$AA_?$AAI?$AAn?$AAt?$AAe?$AAr?$AAn?$AAa?$AAl?$AAM?$AAa?$AAp?$AAR?$AAe?$AAg?$AAi?$AAs?$AAt?$AAe?$AAr?$AAA?$AAd?$AAd?$AAr?$AAe?$AAs?$AAs?$AAe@ 10001f10     sim_common_topaz_v1:simhw.obj
 0001:00000f58       ??_C@_1FE@MEMJELON@?$AAS?$AAI?$AAM?$AA_?$AAI?$AAn?$AAt?$AAe?$AAr?$AAn?$AAa?$AAl?$AAM?$AAa?$AAp?$AAR?$AAe?$AAg?$AAi?$AAs?$AAt?$AAe?$AAr?$AAA?$AAd?$AAd?$AAr?$AAe?$AAs?$AAs?$AAe?$AAs@ 10001f58     sim_common_topaz_v1:simhw.obj
 0001:00000fb0       ??_C@_1EG@OCMGIJKB@?$AA?$CL?$AAS?$AAI?$AAM?$AA_?$AAI?$AAn?$AAt?$AAe?$AAr?$AAn?$AAa?$AAl?$AAM?$AAa?$AAp?$AAR?$AAe?$AAg?$AAi?$AAs?$AAt?$AAe?$AAr?$AAA?$AAd?$AAd?$AAr?$AAe?$AAs?$AAs?$AAe@ 10001fb0     sim_common_topaz_v1:simhw.obj
 0001:00000ff8       ??_C@_1EK@PBCLMPFE@?$AA?9?$AAS?$AAI?$AAM?$AA_?$AAI?$AAn?$AAt?$AAe?$AAr?$AAn?$AAa?$AAl?$AAU?$AAn?$AAM?$AAa?$AAp?$AAR?$AAe?$AAg?$AAi?$AAs?$AAt?$AAe?$AAr?$AAA?$AAd?$AAd?$AAr?$AAe?$AAs@ 10001ff8     sim_common_topaz_v1:simhw.obj
 0001:00001048       ??_C@_1EK@MPBIICEN@?$AA?$CL?$AAS?$AAI?$AAM?$AA_?$AAI?$AAn?$AAt?$AAe?$AAr?$AAn?$AAa?$AAl?$AAU?$AAn?$AAM?$AAa?$AAp?$AAR?$AAe?$AAg?$AAi?$AAs?$AAt?$AAe?$AAr?$AAA?$AAd?$AAd?$AAr?$AAe?$AAs@ 10002048     sim_common_topaz_v1:simhw.obj
 0001:00001094       ??_C@_1BG@BBHPEFCB@?$AA?9?$AAS?$AAI?$AAM?$AA_?$AAI?$AAn?$AAi?$AAt?$AA?6?$AA?$AA@ 10002094     sim_common_topaz_v1:simhw.obj
 0001:000010b0       ??_C@_1FK@POMEHCGJ@?$AAI?$AAs?$AAr?$AAT?$AAh?$AAr?$AAe?$AAa?$AAd?$AAP?$AAr?$AAo?$AAc?$AA?3?$AA?5?$AAK?$AAe?$AAy?$AAb?$AAd?$AAI?$AAn?$AAt?$AAe?$AAr?$AAr?$AAu?$AAp?$AAt?$AAE?$AAn?$AAa@ 100020b0     sim_common_topaz_v1:simhw.obj
 0001:00001110       ??_C@_1HG@EMHCHOG@?$AAE?$AAR?$AAR?$AAO?$AAR?$AA?3?$AA?5?$AAF?$AAa?$AAi?$AAl?$AAe?$AAd?$AA?5?$AAt?$AAo?$AA?5?$AAo?$AAb?$AAt?$AAa?$AAi?$AAn?$AA?5?$AAs?$AAy?$AAs?$AAi?$AAn?$AAt?$AAr?$AA?5@ 10002110     sim_common_topaz_v1:simhw.obj
 0001:00001188       ??_C@_1HG@PGIJENLL@?$AAE?$AAR?$AAR?$AAO?$AAR?$AA?3?$AA?5?$AAF?$AAa?$AAi?$AAl?$AAe?$AAd?$AA?5?$AAt?$AAo?$AA?5?$AAg?$AAe?$AAt?$AA?5?$AAt?$AAh?$AAe?$AA?5?$AAl?$AAi?$AAs?$AAt?$AA?5?$AAo?$AAf@ 10002188     sim_common_topaz_v1:simhw.obj
 0001:00001200       ??_C@_1GG@OANEJLPK@?$AAE?$AAR?$AAR?$AAO?$AAR?$AA?3?$AA?5?$AAF?$AAa?$AAi?$AAl?$AAe?$AAd?$AA?5?$AAt?$AAo?$AA?5?$AAc?$AAr?$AAe?$AAa?$AAt?$AAe?$AA?5?$AAe?$AAv?$AAe?$AAn?$AAt?$AA?5?$AAf?$AAo@ 10002200     sim_common_topaz_v1:simhw.obj
 0001:00001268       ??_C@_1BG@GDIOBPKB@?$AA?$CL?$AAS?$AAI?$AAM?$AA_?$AAI?$AAn?$AAi?$AAt?$AA?6?$AA?$AA@ 10002268     sim_common_topaz_v1:simhw.obj
 0001:00001280       ??_C@_1BG@DCMHGFCI@?$AA?9?$AAS?$AAI?$AAM?$AA_?$AAO?$AAp?$AAe?$AAn?$AA?6?$AA?$AA@ 10002280     sim_common_topaz_v1:simhw.obj
 0001:00001298       ??_C@_1FM@IKHPMKLK@?$AAS?$AAI?$AAM?$AA_?$AAO?$AAp?$AAe?$AAn?$AA?3?$AA?5?$AA?5?$AAB?$AAS?$AAP?$AAS?$AAe?$AAt?$AAS?$AAI?$AAM?$AAC?$AAl?$AAo?$AAc?$AAk?$AAG?$AAa?$AAt?$AAi?$AAn?$AAg?$AAM@ 10002298     sim_common_topaz_v1:simhw.obj
 0001:000012f4       ??_C@_1CI@OHCJFJPM@?$AAE?$AAR?$AAR?$AAO?$AAR?$AA?3?$AA?5?$AA?$CF?$AAs?$AA?5?$AAl?$AAi?$AAn?$AAe?$AA?5?$AA?$CF?$AAd?$AA?3?$AA?5?$AA?$AA@ 100022f4     sim_common_topaz_v1:simhw.obj
 0001:00001320       ??_C@_1KG@MOAJPAJC@?$AAC?$AA?3?$AA?2?$AAW?$AAI?$AAN?$AAC?$AAE?$AAR?$AAO?$AAO?$AAT?$AAS?$AA?2?$AAT?$AAo?$AAp?$AAa?$AAz?$AA?2?$AAW?$AAI?$AAN?$AAC?$AAE?$AA6?$AA0?$AA0?$AA?2?$AAP?$AAL?$AAA@ 10002320     sim_common_topaz_v1:simhw.obj
 0001:000013c8       ??_C@_1BG@EADGDPKI@?$AA?$CL?$AAS?$AAI?$AAM?$AA_?$AAO?$AAp?$AAe?$AAn?$AA?6?$AA?$AA@ 100023c8     sim_common_topaz_v1:simhw.obj
 0001:000013e0       ??_C@_1BI@CFOBNBDC@?$AA?9?$AAS?$AAI?$AAM?$AA_?$AAC?$AAl?$AAo?$AAs?$AAe?$AA?6?$AA?$AA@ 100023e0     sim_common_topaz_v1:simhw.obj
 0001:000013f8       ??_C@_1BI@JFNMIDGC@?$AA?$CL?$AAS?$AAI?$AAM?$AA_?$AAC?$AAl?$AAo?$AAs?$AAe?$AA?6?$AA?$AA@ 100023f8     sim_common_topaz_v1:simhw.obj
 0001:00001410       ??_C@_1CA@KODCEABL@?$AA?9?$AAS?$AAI?$AAM?$AA_?$AAC?$AAo?$AAl?$AAd?$AAR?$AAe?$AAs?$AAe?$AAt?$AA?6?$AA?$AA@ 10002410     sim_common_topaz_v1:simhw.obj
 0001:00001430       ??_C@_1BE@MBFBFCJE@?$AAL?$AAR?$AAC?$AA?5?$AAE?$AAr?$AAr?$AAo?$AAr?$AA?$AA@ 10002430     sim_common_topaz_v1:simhw.obj
 0001:00001444       ??_C@_1BM@LILBCNI@?$AAC?$AAW?$AAT?$AA?5?$AAT?$AAi?$AAm?$AAe?$AAO?$AAu?$AAt?$AA?$AN?$AA?6?$AA?$AA@ 10002444     sim_common_topaz_v1:simhw.obj
 0001:00001460       ??_C@_1CE@BCBOPDPG@?$AAG?$AAP?$AAC?$AAO?$AAU?$AAN?$AAT?$AA?5?$AAT?$AAi?$AAm?$AAe?$AAO?$AAu?$AAt?$AA?$AN?$AA?6?$AA?$AA@ 10002460     sim_common_topaz_v1:simhw.obj
 0001:00001488       ??_C@_1GA@DNAGIHML@?$AAS?$AAI?$AAM?$AA?5?$AAR?$AAE?$AAC?$AAV?$AA?5?$AAi?$AAn?$AAt?$AAe?$AAr?$AAr?$AAu?$AAp?$AAt?$AA?5?$AAt?$AAi?$AAm?$AAe?$AA?5?$AAo?$AAu?$AAt?$AA?$CB?$AAR?$AAC?$AAV?$AA?3@ 10002488     sim_common_topaz_v1:simhw.obj
 0001:000014e8       ??_C@_1CM@HMENDFPC@?$AAG?$AAP?$AAC?$AAN?$AAT?$AA?5?$AAt?$AAi?$AAm?$AAe?$AA?5?$AAo?$AAu?$AAt?$AA?$CB?$AA0?$AAx?$AA?$CF?$AAx?$AA?$AN?$AA?6?$AA?$AA@ 100024e8     sim_common_topaz_v1:simhw.obj
 0001:00001514       ??_C@_1CA@OHHNFHCE@?$AA?$CL?$AAS?$AAI?$AAM?$AA_?$AAC?$AAo?$AAl?$AAd?$AAR?$AAe?$AAs?$AAe?$AAt?$AA?6?$AA?$AA@ 10002514     sim_common_topaz_v1:simhw.obj
 0001:00001534       ??_C@_1CA@KIGJJCHC@?$AA?9?$AAS?$AAI?$AAM?$AA_?$AAW?$AAa?$AAr?$AAm?$AAR?$AAe?$AAs?$AAe?$AAt?$AA?6?$AA?$AA@ 10002534     sim_common_topaz_v1:simhw.obj
 0001:00001554       ??_C@_1DE@ODOJKBMP@?$AAG?$AAP?$AAC?$AAN?$AAT?$AA?5?$AAt?$AAi?$AAm?$AAe?$AA?5?$AAo?$AAu?$AAt?$AA?5?$AA?$CI?$AA2?$AA?$CJ?$AA?$CB?$AA0?$AAx?$AA?$CF?$AAx?$AA?$AN?$AA?6?$AA?$AA@ 10002554     sim_common_topaz_v1:simhw.obj
 0001:00001588       ??_C@_1DE@EMEAOMAF@?$AAG?$AAP?$AAC?$AAN?$AAT?$AA?5?$AAt?$AAi?$AAm?$AAe?$AA?5?$AAo?$AAu?$AAt?$AA?5?$AA?$CI?$AA1?$AA?$CJ?$AA?$CB?$AA0?$AAx?$AA?$CF?$AAx?$AA?$AN?$AA?6?$AA?$AA@ 10002588     sim_common_topaz_v1:simhw.obj
 0001:000015bc       ??_C@_1CA@OBCGIFEN@?$AA?$CL?$AAS?$AAI?$AAM?$AA_?$AAW?$AAa?$AAr?$AAm?$AAR?$AAe?$AAs?$AAe?$AAt?$AA?6?$AA?$AA@ 100025bc     sim_common_topaz_v1:simhw.obj
 0001:000015dc       ??_C@_1BO@NNKBHBHB@?$AA?9?$AAS?$AAI?$AAM?$AA_?$AAR?$AAe?$AAa?$AAd?$AAD?$AAa?$AAt?$AAa?$AA?6?$AA?$AA@ 100025dc     sim_common_topaz_v1:simhw.obj
 0001:000015fc       ??_C@_1DA@MBCNLDGH@?$AAC?$AAW?$AAT?$AA?5?$AAT?$AAi?$AAm?$AAe?$AAO?$AAu?$AAt?$AA?5?$AAi?$AAn?$AA?5?$AAS?$AAI?$AAM?$AA_?$AAR?$AAe?$AAa?$AAd?$AA?$AA@ 100025fc     sim_common_topaz_v1:simhw.obj
 0001:00001630       ??_C@_1GK@IGFFFNBP@?$AAS?$AAI?$AAM?$AA?5?$AAr?$AAe?$AAa?$AAd?$AA?5?$AAd?$AAa?$AAt?$AAa?$AA?5?$AAi?$AAn?$AAt?$AAe?$AAr?$AAr?$AAu?$AAp?$AAt?$AA?5?$AAt?$AAi?$AAm?$AAe?$AA?5?$AAo?$AAu?$AAt@ 10002630     sim_common_topaz_v1:simhw.obj
 0001:0000169c       ??_C@_1BO@FEODDLEB@?$AA?$CL?$AAS?$AAI?$AAM?$AA_?$AAR?$AAe?$AAa?$AAd?$AAD?$AAa?$AAt?$AAa?$AA?6?$AA?$AA@ 1000269c     sim_common_topaz_v1:simhw.obj
 0001:000016bc       ??_C@_1CA@ICPAOBAA@?$AA?9?$AAS?$AAI?$AAM?$AA_?$AAW?$AAr?$AAi?$AAt?$AAe?$AAD?$AAa?$AAt?$AAa?$AA?6?$AA?$AA@ 100026bc     sim_common_topaz_v1:simhw.obj
 0001:000016e0       ??_C@_1GM@IKPOPNPO@?$AAS?$AAI?$AAM?$AA?5?$AAw?$AAr?$AAi?$AAt?$AAe?$AA?5?$AAd?$AAa?$AAt?$AAa?$AA?5?$AAi?$AAn?$AAt?$AAe?$AAr?$AAr?$AAu?$AAp?$AAt?$AA?5?$AAt?$AAi?$AAm?$AAe?$AA?5?$AAo?$AAu@ 100026e0     sim_common_topaz_v1:simhw.obj
 0001:0000174c       ??_C@_1CA@MLLPPGDP@?$AA?$CL?$AAS?$AAI?$AAM?$AA_?$AAW?$AAr?$AAi?$AAt?$AAe?$AAD?$AAa?$AAt?$AAa?$AA?6?$AA?$AA@ 1000274c     sim_common_topaz_v1:simhw.obj
 0001:0000176c       ??_C@_1CC@EHJCPJDD@?$AA?9?$AAS?$AAI?$AAM?$AA_?$AAD?$AAe?$AAa?$AAc?$AAt?$AAi?$AAv?$AAa?$AAt?$AAe?$AA?6?$AA?$AA@ 1000276c     sim_common_topaz_v1:simhw.obj
 0001:00001790       ??_C@_1CC@JMJPBPIH@?$AA?$CL?$AAS?$AAI?$AAM?$AA_?$AAD?$AAe?$AAa?$AAc?$AAt?$AAi?$AAv?$AAa?$AAt?$AAe?$AA?6?$AA?$AA@ 10002790     sim_common_topaz_v1:simhw.obj
 0001:000017b4       ??_C@_1CA@FPHFKBAA@?$AA?9?$AAS?$AAI?$AAM?$AA_?$AAC?$AAo?$AAn?$AAf?$AAi?$AAg?$AAC?$AAL?$AAK?$AA?6?$AA?$AA@ 100027b4     sim_common_topaz_v1:simhw.obj
 0001:000017d4       ??_C@_1DC@BOAKCEJK@?$AAC?$AAu?$AAr?$AAr?$AAe?$AAn?$AAt?$AA?5?$AAb?$AAa?$AAu?$AAd?$AA?5?$AAr?$AAa?$AAt?$AAe?$AA?5?$AA?3?$AA?5?$AA?$CF?$AAd?$AA?$AN?$AA?6?$AA?$AA@ 100027d4     sim_common_topaz_v1:simhw.obj
 0001:00001808       ??_C@_1DI@JCACKPDH@?$AAU?$AAn?$AAs?$AAu?$AAp?$AAp?$AAo?$AAr?$AAt?$AAe?$AAd?$AA?5?$AAC?$AAL?$AAK?$AA_?$AAP?$AAR?$AAE?$AAS?$AAC?$AAA?$AAL?$AAE?$AAR?$AA?$AN?$AA?6?$AA?$AA@ 10002808     sim_common_topaz_v1:simhw.obj
 0001:00001840       ??_C@_1DI@GJOJIKKO@?$AAf?$AAr?$AAe?$AAp?$AA?3?$AA?$CF?$AAd?$AA?5?$AA?$DN?$AA?5?$AA?$CF?$AAd?$AA?5?$AAM?$AAH?$AAz?$AA?5?$AA?1?$AA?5?$AA?$CF?$AAd?$AA?5?$AAM?$AAH?$AAz?$AA?$AN?$AA?6?$AA?$AA@ 10002840     sim_common_topaz_v1:simhw.obj
 0001:00001878       ??_C@_1CO@ICBBAAKK@?$AAU?$AAn?$AAs?$AAu?$AAp?$AAp?$AAo?$AAr?$AAt?$AAe?$AAd?$AA?5?$AAf?$AA?5?$AA?3?$AA?5?$AA?$CF?$AA0?$AA2?$AAx?$AA?$AN?$AA?6?$AA?$AA@ 10002878     sim_common_topaz_v1:simhw.obj
 0001:000018a8       ??_C@_1CK@DCGMODMI@?$AAU?$AAn?$AAs?$AAu?$AAp?$AAp?$AAo?$AAr?$AAt?$AAe?$AAd?$AA?5?$AAf?$AA?5?$AA?3?$AA?5?$AA?$CF?$AAd?$AA?$AN?$AA?6?$AA?$AA@ 100028a8     sim_common_topaz_v1:simhw.obj
 0001:000018d4       ??_C@_1CA@BGDKLGDP@?$AA?$CL?$AAS?$AAI?$AAM?$AA_?$AAC?$AAo?$AAn?$AAf?$AAi?$AAg?$AAC?$AAL?$AAK?$AA?6?$AA?$AA@ 100028d4     sim_common_topaz_v1:simhw.obj
 0001:000018f4       ??_C@_1CC@NJCDDGNG@?$AA?9?$AAS?$AAI?$AAM?$AA_?$AAC?$AAo?$AAn?$AAf?$AAi?$AAg?$AAT?$AAi?$AAm?$AAe?$AA?6?$AA?$AA@ 100028f4     sim_common_topaz_v1:simhw.obj
 0001:00001918       ??_C@_1CC@CCONAGC@?$AA?$CL?$AAS?$AAI?$AAM?$AA_?$AAC?$AAo?$AAn?$AAf?$AAi?$AAg?$AAT?$AAi?$AAm?$AAe?$AA?6?$AA?$AA@ 10002918     sim_common_topaz_v1:simhw.obj
 0001:0000193c       ??_C@_1BO@KOALDFJO@?$AAS?$AAI?$AAM?$AA_?$AAC?$AAh?$AAe?$AAc?$AAk?$AAC?$AAa?$AAr?$AAd?$AA?6?$AA?$AA@ 1000293c     sim_common_topaz_v1:simhw.obj
 0001:0000195c       ??_C@_1CK@MLMNBOHC@?$AA?9?$AAS?$AAI?$AAM?$AA_?$AAM?$AAa?$AAs?$AAk?$AAI?$AAn?$AAt?$AAe?$AAr?$AAr?$AAu?$AAp?$AAt?$AAs?$AA?6?$AA?$AA@ 1000295c     sim_common_topaz_v1:simhw.obj
 0001:00001988       ??_C@_1CK@LLLKAIJE@?$AA?$CL?$AAS?$AAI?$AAM?$AA_?$AAM?$AAa?$AAs?$AAk?$AAI?$AAn?$AAt?$AAe?$AAr?$AAr?$AAu?$AAp?$AAt?$AAs?$AA?6?$AA?$AA@ 10002988     sim_common_topaz_v1:simhw.obj
 0001:000019b4       ??_C@_1CA@PHLHGPAC@?$AA?9?$AAS?$AAI?$AAM?$AA_?$AAF?$AAl?$AAu?$AAs?$AAh?$AAF?$AAI?$AAF?$AAO?$AA?6?$AA?$AA@ 100029b4     sim_common_topaz_v1:simhw.obj
 0001:000019d4       ??_C@_1CA@LOPIHIDN@?$AA?$CL?$AAS?$AAI?$AAM?$AA_?$AAF?$AAl?$AAu?$AAs?$AAh?$AAF?$AAI?$AAF?$AAO?$AA?6?$AA?$AA@ 100029d4     sim_common_topaz_v1:simhw.obj
 0001:000019f4       ??_C@_1BG@HPGECGNM@?$AAB?$AAG?$AAT?$AA?3?$AA?5?$AA?$CF?$AAx?$AA?5?$AA?$AN?$AA?6?$AA?$AA@ 100029f4     sim_common_topaz_v1:simhw.obj
 0001:00001a0c       ??_C@_1BG@JPKCINPJ@?$AAB?$AAW?$AAT?$AA?3?$AA?5?$AA?$CF?$AAx?$AA?5?$AA?$AN?$AA?6?$AA?$AA@ 10002a0c     sim_common_topaz_v1:simhw.obj
 0001:00001a24       ??_C@_1BO@NOCNBALG@?$AAD?$AAi?$AAv?$AAi?$AAs?$AAo?$AAr?$AA?3?$AA?5?$AA?$CF?$AAx?$AA?5?$AA?$AN?$AA?6?$AA?$AA@ 10002a24     sim_common_topaz_v1:simhw.obj
 0001:00001a44       ??_C@_1BO@MLFMICDK@?$AAG?$AAP?$AAC?$AAO?$AAU?$AAN?$AAT?$AA?3?$AA?5?$AA?$CF?$AAx?$AA?5?$AA?$AN?$AA?6?$AA?$AA@ 10002a44     sim_common_topaz_v1:simhw.obj
 0001:00001a64       ??_C@_1CC@CDEENKEM@?$AAC?$AAh?$AAa?$AAr?$AA_?$AAW?$AAa?$AAi?$AAt?$AA?3?$AA?5?$AA?$CF?$AAx?$AA?5?$AA?$AN?$AA?6?$AA?$AA@ 10002a64     sim_common_topaz_v1:simhw.obj
 0001:00001a88       ??_C@_1CK@NDDNLBCG@?$AAR?$AAe?$AAs?$AAe?$AAt?$AA_?$AAC?$AAo?$AAn?$AAt?$AAr?$AAo?$AAl?$AA?3?$AA?5?$AA?$CF?$AAx?$AA?5?$AA?$AN?$AA?6?$AA?$AA@ 10002a88     sim_common_topaz_v1:simhw.obj
 0001:00001ab4       ??_C@_1CC@CJPMFIN@?$AAO?$AAD?$AA_?$AAC?$AAO?$AAN?$AAF?$AAI?$AAG?$AA?3?$AA?5?$AA?$CF?$AAx?$AA?5?$AA?$AN?$AA?6?$AA?$AA@ 10002ab4     sim_common_topaz_v1:simhw.obj
 0001:00001ad8       ??_C@_1CE@EPPBDPLN@?$AAG?$AAu?$AAa?$AAr?$AAd?$AA_?$AAC?$AAn?$AAt?$AAl?$AA?3?$AA?5?$AA?$CF?$AAx?$AA?5?$AA?$AN?$AA?6?$AA?$AA@ 10002ad8     sim_common_topaz_v1:simhw.obj
 0001:00001afc       ??_C@_1CK@HPLELPFL@?$AAX?$AAm?$AAt?$AA_?$AAt?$AAh?$AAr?$AAe?$AAs?$AAh?$AAo?$AAl?$AAd?$AA?3?$AA?5?$AA?$CF?$AAx?$AA?5?$AA?$AN?$AA?6?$AA?$AA@ 10002afc     sim_common_topaz_v1:simhw.obj
 0001:00001b28       ??_C@_1CG@GGKHDDKE@?$AAD?$AAa?$AAt?$AAa?$AA_?$AAF?$AAo?$AAr?$AAm?$AAa?$AAt?$AA?3?$AA?5?$AA?$CF?$AAx?$AA?5?$AA?$AN?$AA?6?$AA?$AA@ 10002b28     sim_common_topaz_v1:simhw.obj
 0001:00001b50       ??_C@_1CI@FEEJHKCF@?$AAp?$AAo?$AAr?$AAt?$AA0?$AA_?$AAd?$AAe?$AAt?$AAe?$AAc?$AAt?$AA?3?$AA?5?$AA?$CF?$AAx?$AA?5?$AA?$AN?$AA?6?$AA?$AA@ 10002b50     sim_common_topaz_v1:simhw.obj
 0001:00001b78       ??_C@_1CA@CGGFJFIP@?$AAI?$AAn?$AAt?$AA_?$AAm?$AAa?$AAs?$AAk?$AA?3?$AA?5?$AA?$CF?$AAx?$AA?5?$AA?$AN?$AA?6?$AA?$AA@ 10002b78     sim_common_topaz_v1:simhw.obj
 0001:00001b98       ??_C@_1CE@GILGDIFJ@?$AAR?$AAx?$AAv?$AA_?$AAs?$AAt?$AAa?$AAt?$AAu?$AAs?$AA?3?$AA?5?$AA?$CF?$AAx?$AA?5?$AA?$AN?$AA?6?$AA?$AA@ 10002b98     sim_common_topaz_v1:simhw.obj
 0001:00001bbc       ??_C@_1CG@PMJIAFIK@?$AAT?$AAx?$AAm?$AAt?$AA_?$AAs?$AAt?$AAa?$AAt?$AAu?$AAs?$AA?3?$AA?5?$AA?$CF?$AAx?$AA?5?$AA?$AN?$AA?6?$AA?$AA@ 10002bbc     sim_common_topaz_v1:simhw.obj
 0001:00001be4       ??_C@_1CC@CKAMHIDN@?$AAE?$AAn?$AAa?$AAb?$AAl?$AAe?$AAR?$AAe?$AAg?$AA?3?$AA?5?$AA?$CF?$AAx?$AA?5?$AA?$AN?$AA?6?$AA?$AA@ 10002be4     sim_common_topaz_v1:simhw.obj
 0001:00001c08       ??_C@_1DC@DHIHIMEM@?$AAr?$AAe?$AAc?$AAi?$AAe?$AAv?$AAe?$AA_?$AAt?$AAh?$AAr?$AAe?$AAs?$AAh?$AAo?$AAl?$AAd?$AA?3?$AA?5?$AA?$CF?$AAx?$AA?5?$AA?$AN?$AA?6?$AA?$AA@ 10002c08     sim_common_topaz_v1:simhw.obj
 0001:00001c3c       ??_C@_1CI@PEJPJCFD@?$AAc?$AAl?$AAc?$AAo?$AAk?$AA_?$AAs?$AAe?$AAl?$AAe?$AAc?$AAt?$AA?3?$AA?5?$AA?$CF?$AAx?$AA?5?$AA?$AN?$AA?6?$AA?$AA@ 10002c3c     sim_common_topaz_v1:simhw.obj
 0001:00001c64       ??_C@_1CO@KKDAIACC@?$AAC?$AAo?$AAn?$AAt?$AAr?$AAo?$AAl?$AAR?$AAe?$AAg?$AAi?$AAs?$AAt?$AAe?$AAr?$AA?3?$AA?5?$AA?$CF?$AAx?$AA?5?$AA?$AN?$AA?6?$AA?$AA@ 10002c64     sim_common_topaz_v1:simhw.obj
 0001:00001c94       ??_C@_1CE@KLAHDILH@?$AAp?$AAo?$AAr?$AAt?$AA0?$AA_?$AAc?$AAn?$AAt?$AAl?$AA?3?$AA?5?$AA?$CF?$AAx?$AA?5?$AA?$AN?$AA?6?$AA?$AA@ 10002c94     sim_common_topaz_v1:simhw.obj
 0001:00001cb8       ??_C@_1CG@DJPPOLPP@?$AAp?$AAo?$AAr?$AAt?$AA1?$AAd?$AAe?$AAt?$AAe?$AAc?$AAt?$AA?3?$AA?5?$AA?$CF?$AAx?$AA?5?$AA?$AN?$AA?6?$AA?$AA@ 10002cb8     sim_common_topaz_v1:simhw.obj
 0001:00001ce0       ??_C@_1CK@OKNEOHBG@?$AAS?$AAe?$AAt?$AAu?$AAp?$AAR?$AAe?$AAg?$AAi?$AAs?$AAt?$AAe?$AAr?$AA?3?$AA?5?$AA?$CF?$AAx?$AA?5?$AA?$AN?$AA?6?$AA?$AA@ 10002ce0     sim_common_topaz_v1:simhw.obj
 0001:00001d0c       ??_C@_1CE@KKLCMFKK@?$AAp?$AAo?$AAr?$AAt?$AA1?$AA_?$AAc?$AAn?$AAt?$AAl?$AA?3?$AA?5?$AA?$CF?$AAx?$AA?5?$AA?$AN?$AA?6?$AA?$AA@ 10002d0c     sim_common_topaz_v1:simhw.obj
 0001:00001d30       NTStatusC000Table          10002d30     smclib:smcce.obj
 0001:000022c0       NTStatus8000Table          100032c0     smclib:smcce.obj
 0001:00002310       ??_C@_1GK@JMBHNEDO@?$AA?$CF?$AAs?$AA?$CB?$AAS?$AAm?$AAa?$AAr?$AAt?$AAc?$AAa?$AAr?$AAd?$AAC?$AAr?$AAe?$AAa?$AAt?$AAe?$AAL?$AAi?$AAn?$AAk?$AA?3?$AA?5?$AA?$FL?$AA?$CF?$AAs?$AA?$FN?$AA?5?$AA?9?$AA?$DO?$AA?5@ 10003310     smclib:smcce.obj
 0001:0000237c       ??_C@_06LAPNJEMN@SMCLIB?$AA@ 1000337c     smclib:smcce.obj
 0001:00002384       ??_C@_1CG@HNJJIDPF@?$AAS?$AAC?$AAa?$AAr?$AAd?$AAF?$AAo?$AAr?$AAg?$AAe?$AAt?$AAR?$AAe?$AAa?$AAd?$AAe?$AAr?$AAW?$AA?$AA@ 10003384     smclib:smcce.obj
 0001:000023ac       ??_C@_1CM@MEAEFIBF@?$AAS?$AAC?$AAa?$AAr?$AAd?$AAI?$AAn?$AAt?$AAr?$AAo?$AAd?$AAu?$AAc?$AAe?$AAR?$AAe?$AAa?$AAd?$AAe?$AAr?$AAW?$AA?$AA@ 100033ac     smclib:smcce.obj
 0001:000023d8       ??_C@_1BK@JIMBCHBC@?$AAW?$AAI?$AAN?$AAS?$AAC?$AAA?$AAR?$AAD?$AA?4?$AAD?$AAL?$AAL?$AA?$AA@ 100033d8     smclib:smcce.obj
 0001:000023f8       ??_C@_1FK@KGECNCKA@?$AA?$CF?$AAs?$AA?$CB?$AAS?$AAm?$AAa?$AAr?$AAt?$AAc?$AAa?$AAr?$AAd?$AAD?$AAe?$AAl?$AAe?$AAt?$AAe?$AAL?$AAi?$AAn?$AAk?$AA?3?$AA?5?$AA?$FL?$AA?$CF?$AAs?$AA?$FN?$AA?5?$AA?0?$AA?5?$AAs@ 100033f8     smclib:smcce.obj
 0001:00002454       ??_C@_1DM@FLECFOAI@?$AA?$CF?$AAs?$AA?$CB?$AAS?$AAm?$AAa?$AAr?$AAt?$AAc?$AAa?$AAr?$AAd?$AAI?$AAn?$AAi?$AAt?$AAi?$AAa?$AAl?$AAi?$AAz?$AAe?$AA?3?$AA?5?$AAE?$AAx?$AAi?$AAt?$AA?6?$AA?$AA@ 10003454     smclib:smcce.obj
 0001:00002490       ??_C@_1LE@LLONJMAA@?$AA?$CF?$AAs?$AA?$CB?$AAS?$AAm?$AAa?$AAr?$AAt?$AAc?$AAa?$AAr?$AAd?$AAI?$AAn?$AAi?$AAt?$AAi?$AAa?$AAl?$AAi?$AAz?$AAe?$AA?3?$AA?5?$AAW?$AAA?$AAR?$AAN?$AAI?$AAN?$AAG?$AA?3@ 10003490     smclib:smcce.obj
 0001:00002548       ??_C@_1LI@GLGCLFHC@?$AA?$CF?$AAs?$AA?$CB?$AAS?$AAm?$AAa?$AAr?$AAt?$AAc?$AAa?$AAr?$AAd?$AAI?$AAn?$AAi?$AAt?$AAi?$AAa?$AAl?$AAi?$AAz?$AAe?$AA?3?$AA?5?$AAW?$AAA?$AAR?$AAN?$AAI?$AAN?$AAG?$AA?3@ 10003548     smclib:smcce.obj
 0001:00002600       ??_C@_1IM@DBDMEFND@?$AA?$CF?$AAs?$AA?$CB?$AAS?$AAm?$AAa?$AAr?$AAt?$AAc?$AAa?$AAr?$AAd?$AAI?$AAn?$AAi?$AAt?$AAi?$AAa?$AAl?$AAi?$AAz?$AAe?$AA?3?$AA?5?$AAI?$AAn?$AAc?$AAo?$AAm?$AAp?$AAa?$AAt@ 10003600     smclib:smcce.obj
 0001:00002690       ??_C@_1IC@ONAEBHFJ@?$AAD?$AA?3?$AA?2?$AAy?$AAa?$AAm?$AAa?$AAf?$AAp?$AA?9?$AA1?$AA?2?$AAp?$AAu?$AAb?$AAl?$AAi?$AAc?$AA?2?$AAC?$AAO?$AAM?$AAM?$AAO?$AAN?$AA?2?$AAo?$AAa?$AAk?$AA?2?$AAd?$AAr@ 10003690     smclib:smcce.obj
 0001:00002718       ??_C@_1GG@BBMMIPNJ@?$AA?$CF?$AAs?$AA?$CB?$AAS?$AAm?$AAa?$AAr?$AAt?$AAc?$AAa?$AAr?$AAd?$AAI?$AAn?$AAi?$AAt?$AAi?$AAa?$AAl?$AAi?$AAz?$AAe?$AA?3?$AA?5?$AAE?$AAn?$AAt?$AAe?$AAr?$AA?4?$AA?5?$AAV@ 10003718     smclib:smcce.obj
 0001:00002780       ??_C@_0M@KBNPCODE@Sep?530?52007?$AA@ 10003780     smclib:smcce.obj
 0001:0000278c       ??_C@_08LHJNAMGL@22?341?330?$AA@ 1000378c     smclib:smcce.obj
 0001:00002798       ??_C@_1DA@MAGKCMH@?$AA?$CF?$AAs?$AA?$CB?$AAS?$AAm?$AAa?$AAr?$AAt?$AAc?$AAa?$AAr?$AAd?$AAE?$AAx?$AAi?$AAt?$AA?3?$AA?5?$AAE?$AAx?$AAi?$AAt?$AA?6?$AA?$AA@ 10003798     smclib:smcce.obj
 0001:000027c8       ??_C@_1DC@LFMLJDHC@?$AA?$CF?$AAs?$AA?$CB?$AAS?$AAm?$AAa?$AAr?$AAt?$AAc?$AAa?$AAr?$AAd?$AAE?$AAx?$AAi?$AAt?$AA?3?$AA?5?$AAE?$AAn?$AAt?$AAe?$AAr?$AA?6?$AA?$AA@ 100037c8     smclib:smcce.obj
 0001:00002800       ??_C@_1EG@CJOIFBJL@?$AA?$CF?$AAs?$AA?$CB?$AA?$CI?$AAS?$AAm?$AAa?$AAr?$AAt?$AAc?$AAa?$AAr?$AAd?$AAD?$AAe?$AAv?$AAi?$AAc?$AAe?$AAC?$AAo?$AAn?$AAt?$AAr?$AAo?$AAl?$AA?$CJ?$AA?3?$AA?5?$AAE?$AAx?$AAi@ 10003800     smclib:smcce.obj
 0001:00002848       ??_C@_1FO@DGBBOPIP@?$AA?$CF?$AAs?$AA?$CB?$AA?$CI?$AAC?$AAo?$AAm?$AAp?$AAl?$AAe?$AAt?$AAi?$AAn?$AAg?$AA?5?$AAI?$AAo?$AAc?$AAt?$AAl?$AA?5?$AA?$DN?$AA?5?$AA?$CF?$AAs?$AA?0?$AA?5?$AAc?$AAu?$AAr?$AAr?$AAe@ 10003848     smclib:smcce.obj
 0001:000028a8       ??_C@_1GE@OCEIDKCK@?$AA?$CF?$AAs?$AA?$CB?$AA?$CI?$AAS?$AAm?$AAa?$AAr?$AAt?$AAc?$AAa?$AAr?$AAd?$AAD?$AAe?$AAv?$AAi?$AAc?$AAe?$AAC?$AAo?$AAn?$AAt?$AAr?$AAo?$AAl?$AA?$CJ?$AA?3?$AA?5?$AAS?$AAy?$AAs@ 100038a8     smclib:smcce.obj
 0001:00002910       ??_C@_1FC@LPNIHAON@?$AA?$CF?$AAs?$AA?$CB?$AA?$CI?$AAS?$AAm?$AAa?$AAr?$AAt?$AAc?$AAa?$AAr?$AAd?$AAD?$AAe?$AAv?$AAi?$AAc?$AAe?$AAC?$AAo?$AAn?$AAt?$AAr?$AAo?$AAl?$AA?$CJ?$AA?3?$AA?5?$AAI?$AAo?$AAc@ 10003910     smclib:smcce.obj
 0001:00002964       ??_C@_13LBAGMAIH@?$AA?6?$AA?$AA@ 10003964     smclib:smcutil.obj
 0001:00002968       ??_C@_1O@OHJNNAJH@?$AA?$CF?$AA0?$AA2?$AAX?$AA?$CF?$AAc?$AA?$AA@ 10003968     smclib:smcutil.obj
 0001:00002978       ??_C@_1IG@KNAFEKIL@?$AAD?$AA?3?$AA?2?$AAy?$AAa?$AAm?$AAa?$AAf?$AAp?$AA?9?$AA1?$AA?2?$AAp?$AAu?$AAb?$AAl?$AAi?$AAc?$AA?2?$AAC?$AAO?$AAM?$AAM?$AAO?$AAN?$AA?2?$AAo?$AAa?$AAk?$AA?2?$AAd?$AAr@ 10003978     smclib:smcutil.obj
 0001:00002a00       ??_C@_1CM@BCHLFIEP@?$AA?5?$AA?5?$AA?5?$AAM?$AAo?$AAd?$AAe?$AA?3?$AA?5?$AAN?$AAe?$AAg?$AAo?$AAt?$AAi?$AAa?$AAb?$AAl?$AAe?$AA?6?$AA?6?$AA?$AA@ 10003a00     smclib:smcutil.obj
 0001:00002a2c       ??_C@_1CO@GBEEFKMP@?$AA?5?$AA?5?$AA?5?$AAM?$AAo?$AAd?$AAe?$AA?3?$AA?5?$AAS?$AAp?$AAe?$AAc?$AAi?$AAf?$AAi?$AAc?$AA?5?$AA?$CF?$AAs?$AA?6?$AA?6?$AA?$AA@ 10003a2c     smclib:smcutil.obj
 0001:00002a5c       ??_C@_11LOCGONAA@?$AA?$AA@ 10003a5c     smclib:smcutil.obj
 0001:00002a60       ??_C@_1BK@DDDLDPG@?$AAs?$AAe?$AAt?$AA?5?$AAb?$AAy?$AA?5?$AAT?$AAA?$AA?$CI?$AA2?$AA?$CJ?$AA?$AA@ 10003a60     smclib:smcutil.obj
 0001:00002a80       ??_C@_1HE@HANNPKHG@?$AA?5?$AA?5?$AA?5?$AAT?$AA?$DN?$AA1?$AA?5?$AAT?$AAi?$AAm?$AAi?$AAn?$AAg?$AA?5?$AAf?$AAr?$AAo?$AAm?$AA?5?$AAA?$AAT?$AAR?$AA?3?$AA?6?$AA?5?$AA?5?$AA?5?$AA?5?$AA?5?$AA?5?$AAC?$AAW@ 10003a80     smclib:smcutil.obj
 0001:00002af8       ??_C@_1JI@EEIAFDAO@?$AA?5?$AA?5?$AA?5?$AAT?$AA?$DN?$AA1?$AA?5?$AAV?$AAa?$AAl?$AAu?$AAe?$AAs?$AA?5?$AAf?$AAr?$AAo?$AAm?$AA?5?$AAA?$AAT?$AAR?$AA?3?$AA?6?$AA?5?$AA?5?$AA?5?$AA?5?$AA?5?$AA?5?$AAI?$AAF@ 10003af8     smclib:smcutil.obj
 0001:00002b90       ??_C@_1FG@OOPEPHLM@?$AA?5?$AA?5?$AA?5?$AAT?$AA?$DN?$AA0?$AA?5?$AAT?$AAi?$AAm?$AAi?$AAn?$AAg?$AA?5?$AAf?$AAr?$AAo?$AAm?$AA?5?$AAA?$AAT?$AAR?$AA?3?$AA?6?$AA?5?$AA?5?$AA?5?$AA?5?$AA?5?$AA?5?$AAW?$AAT@ 10003b90     smclib:smcutil.obj
 0001:00002be8       ??_C@_1FA@CONBDJPM@?$AA?5?$AA?5?$AA?5?$AAT?$AA?$DN?$AA0?$AA?5?$AAV?$AAa?$AAl?$AAu?$AAe?$AAs?$AA?5?$AAf?$AAr?$AAo?$AAm?$AA?5?$AAA?$AAT?$AAR?$AA?3?$AA?6?$AA?5?$AA?5?$AA?5?$AA?5?$AA?5?$AA?5?$AAW?$AAI@ 10003be8     smclib:smcutil.obj
 0001:00002c38       ??_C@_1LC@EPMFJEFM@?$AA?5?$AA?5?$AA?5?$AAC?$AAa?$AAl?$AAc?$AAu?$AAl?$AAa?$AAt?$AAe?$AAd?$AA?5?$AAt?$AAi?$AAm?$AAi?$AAn?$AAg?$AA?5?$AAv?$AAa?$AAl?$AAu?$AAe?$AAs?$AA?3?$AA?6?$AA?5?$AA?5?$AA?5@ 10003c38     smclib:smcutil.obj
 0001:00002cf0       ??_C@_1KM@DPGGHHLG@?$AA?5?$AA?5?$AA?5?$AAP?$AAT?$AAS?$AA?5?$AAp?$AAa?$AAr?$AAa?$AAm?$AAe?$AAt?$AAe?$AAr?$AAs?$AA?5?$AA?$CI?$AA?$CF?$AAs?$AA?$CJ?$AA?3?$AA?6?$AA?5?$AA?5?$AA?5?$AA?5?$AA?5?$AA?5?$AAF?$AAl@ 10003cf0     smclib:smcutil.obj
 0001:00002da0       ??_C@_1MC@LODKHIKL@?$AA?5?$AA?5?$AA?5?$AAC?$AAa?$AAr?$AAd?$AA?5?$AAp?$AAa?$AAr?$AAa?$AAm?$AAe?$AAt?$AAe?$AAr?$AAs?$AA?5?$AAf?$AAr?$AAo?$AAm?$AA?5?$AAA?$AAT?$AAR?$AA?3?$AA?6?$AA?5?$AA?5?$AA?5@ 10003da0     smclib:smcutil.obj
 0001:00002e68       ??_C@_1EG@GMDEFEMG@?$AA?5?$AA?5?$AA?5?$AAD?$AAl?$AA?5?$AA?$DN?$AA?5?$AA?$CF?$AA0?$AA2?$AAx?$AA?5?$AAo?$AAr?$AA?5?$AAF?$AAl?$AA?5?$AA?$DN?$AA?5?$AA?$CF?$AA0?$AA2?$AAx?$AA?5?$AAi?$AAn?$AAv?$AAa?$AAl?$AAi@ 10003e68     smclib:smcutil.obj
 0001:00002eb0       ??_C@_1DO@IJMLPHCG@?$AA?5?$AA?5?$AA?5?$AAA?$AAT?$AAR?$AA?5?$AAl?$AAe?$AAn?$AAg?$AAt?$AAh?$AA?5?$AAi?$AAs?$AA?5?$AAi?$AAn?$AAc?$AAo?$AAn?$AAs?$AAi?$AAs?$AAt?$AAe?$AAn?$AAt?$AA?6?$AA?$AA@ 10003eb0     smclib:smcutil.obj
 0001:00002ef0       ??_C@_1DI@BINOCLOI@?$AA?5?$AA?5?$AA?5?$AAA?$AAT?$AAR?$AA?5?$AAC?$AAh?$AAe?$AAc?$AAk?$AAs?$AAu?$AAm?$AA?5?$AAi?$AAs?$AA?5?$AAi?$AAn?$AAv?$AAa?$AAl?$AAi?$AAd?$AA?6?$AA?$AA@ 10003ef0     smclib:smcutil.obj
 0001:00002f28       ??_C@_1EC@OMJHKKJL@?$AA?5?$AA?5?$AA?5?$AAC?$AAa?$AAr?$AAd?$AA?5?$AAu?$AAs?$AAe?$AAs?$AA?5?$AAI?$AAn?$AAv?$AAe?$AAr?$AAs?$AAe?$AA?5?$AAC?$AAo?$AAn?$AAv?$AAe?$AAn?$AAt?$AAi?$AAo?$AAn?$AA?6@ 10003f28     smclib:smcutil.obj
 0001:00002f70       ??_C@_1FM@GNCIAAEJ@?$AA?5?$AA?5?$AA?5?$AAI?$AAn?$AAi?$AAt?$AAi?$AAa?$AAl?$AA?5?$AAc?$AAh?$AAa?$AAr?$AAa?$AAc?$AAt?$AAe?$AAr?$AA?5?$AA?$CF?$AA0?$AA2?$AAx?$AAh?$AA?5?$AAo?$AAf?$AA?5?$AAA?$AAT@ 10003f70     smclib:smcutil.obj
 0001:00002fcc       ??_C@_1BC@BGBACJME@?$AA?5?$AA?5?$AA?5?$AAA?$AAT?$AAR?$AA?3?$AA?5?$AA?$AA@ 10003fcc     smclib:smcutil.obj
 0001:00002fe0       ??_C@_1FC@DNKICGHA@?$AA?5?$AA?5?$AA?5?$AAA?$AAT?$AAR?$AA?5?$AAi?$AAs?$AA?5?$AAt?$AAo?$AAo?$AA?5?$AAs?$AAh?$AAo?$AAr?$AAt?$AA?5?$AA?$CI?$AAM?$AAi?$AAn?$AA?4?$AA?5?$AAl?$AAe?$AAn?$AAg?$AAt?$AAh@ 10003fe0     smclib:smcutil.obj
 0001:00003038       ??_C@_1EK@OMENJPJJ@?$AA?$CF?$AAs?$AA?$CB?$AAS?$AAm?$AAa?$AAr?$AAt?$AAc?$AAa?$AAr?$AAd?$AAU?$AAp?$AAd?$AAa?$AAt?$AAe?$AAC?$AAa?$AAr?$AAd?$AAC?$AAa?$AAp?$AAa?$AAb?$AAi?$AAl?$AAi?$AAt?$AAi@ 10004038     smclib:smcutil.obj
 0001:00003084       ??_C@_1BM@PNGOEMMA@?$AAP?$AAT?$AAS?$AA_?$AAT?$AAY?$AAP?$AAE?$AA_?$AAU?$AAS?$AAE?$AAR?$AA?$AA@ 10004084     smclib:smcutil.obj
 0001:000030a0       ??_C@_1CC@GLFGFINK@?$AAP?$AAT?$AAS?$AA_?$AAT?$AAY?$AAP?$AAE?$AA_?$AAO?$AAP?$AAT?$AAI?$AAM?$AAA?$AAL?$AA?$AA@ 100040a0     smclib:smcutil.obj
 0001:000030c4       ??_C@_1CC@KGAFFEMB@?$AAP?$AAT?$AAS?$AA_?$AAT?$AAY?$AAP?$AAE?$AA_?$AAD?$AAE?$AAF?$AAA?$AAU?$AAL?$AAT?$AA?$AA@ 100040c4     smclib:smcutil.obj
 0001:000030e8       ??_C@_1NA@BCKMEPIJ@?$AA?$AN?$AA?6?$AA?$CK?$AA?$CK?$AA?$CK?$AA?5?$AAA?$AAS?$AAS?$AAE?$AAR?$AAT?$AAI?$AAO?$AAN?$AA?5?$AAF?$AAA?$AAI?$AAL?$AAE?$AAD?$AA?5?$AAi?$AAn?$AA?5?$AAD?$AA?3?$AA?2?$AAy?$AAa?$AAm@ 100040e8     smclib:smcprot.obj
 0001:000031b8       ??_C@_1PE@MJCMDGMG@?$AA?$AN?$AA?6?$AA?$CK?$AA?$CK?$AA?$CK?$AA?5?$AAA?$AAS?$AAS?$AAE?$AAR?$AAT?$AAI?$AAO?$AAN?$AA?5?$AAF?$AAA?$AAI?$AAL?$AAE?$AAD?$AA?5?$AAi?$AAn?$AA?5?$AAD?$AA?3?$AA?2?$AAy?$AAa?$AAm@ 100041b8     smclib:smcprot.obj
 0001:000032b0       ??_C@_1KE@KFBDEMHG@?$AA?$CF?$AAs?$AA?$CB?$AAS?$AAm?$AAa?$AAr?$AAt?$AAc?$AAa?$AAr?$AAd?$AAT?$AA0?$AAR?$AAe?$AAq?$AAu?$AAe?$AAs?$AAt?$AA?3?$AA?5?$AAL?$AAc?$AA?$CI?$AA?$CF?$AAd?$AA?$CJ?$AA?5?$AAi?$AAn@ 100042b0     smclib:smcprot.obj
 0001:00003358       ??_C@_1JC@OKNJNPCD@?$AA?$CF?$AAs?$AA?$CB?$AAS?$AAm?$AAa?$AAr?$AAt?$AAc?$AAa?$AAr?$AAd?$AAT?$AA0?$AAR?$AAe?$AAq?$AAu?$AAe?$AAs?$AAt?$AA?3?$AA?5?$AAT?$AAP?$AAD?$AAU?$AA?5?$AAi?$AAs?$AA?5?$AAt@ 10004358     smclib:smcprot.obj
 0001:000033f0       ??_C@_1HA@BOMGDFNL@?$AA?$CF?$AAs?$AA?$CB?$AAS?$AAm?$AAa?$AAr?$AAt?$AAc?$AAa?$AAr?$AAd?$AAT?$AA0?$AAR?$AAe?$AAq?$AAu?$AAe?$AAs?$AAt?$AA?3?$AA?5?$AAI?$AAo?$AAR?$AAe?$AAq?$AAu?$AAe?$AAs?$AAt@ 100043f0     smclib:smcprot.obj
 0001:00003460       ??_C@_1NA@KEDFAEON@?$AA?$AN?$AA?6?$AA?$CK?$AA?$CK?$AA?$CK?$AA?5?$AAA?$AAS?$AAS?$AAE?$AAR?$AAT?$AAI?$AAO?$AAN?$AA?5?$AAF?$AAA?$AAI?$AAL?$AAE?$AAD?$AA?5?$AAi?$AAn?$AA?5?$AAD?$AA?3?$AA?2?$AAy?$AAa?$AAm@ 10004460     smclib:smcprot.obj
 0001:00003530       ??_C@_1FM@MDIKABLA@?$AA?$CF?$AAs?$AA?$CB?$AAS?$AAm?$AAa?$AAr?$AAt?$AAc?$AAa?$AAr?$AAd?$AAT?$AA0?$AAR?$AAe?$AAq?$AAu?$AAe?$AAs?$AAt?$AA?3?$AA?5?$AAR?$AAe?$AAp?$AAl?$AAy?$AAB?$AAu?$AAf?$AAf@ 10004530     smclib:smcprot.obj
 0001:00003590       ??_C@_1FC@EDAOCCPG@?$AA?$CF?$AAs?$AA?$CB?$AAS?$AAm?$AAa?$AAr?$AAt?$AAc?$AAa?$AAr?$AAd?$AAT?$AA1?$AAR?$AAe?$AAq?$AAu?$AAe?$AAs?$AAt?$AA?3?$AA?5?$AAI?$AAn?$AAv?$AAa?$AAl?$AAi?$AAd?$AA?5?$AAS@ 10004590     smclib:smcprot.obj
 0001:000035e8       ??_C@_1FA@HFDFCMBC@?$AA?$CF?$AAs?$AA?$CB?$AAS?$AAm?$AAa?$AAr?$AAt?$AAc?$AAa?$AAr?$AAd?$AAT?$AA1?$AAR?$AAe?$AAq?$AAu?$AAe?$AAs?$AAt?$AA?3?$AA?5?$AAT?$AA1?$AA_?$AAW?$AAT?$AAX?$AA_?$AAR?$AAE@ 100045e8     smclib:smcprot.obj
 0001:00003638       ??_C@_1FE@CFCPOKEJ@?$AA?$CF?$AAs?$AA?$CB?$AAS?$AAm?$AAa?$AAr?$AAt?$AAc?$AAa?$AAr?$AAd?$AAT?$AA1?$AAR?$AAe?$AAq?$AAu?$AAe?$AAs?$AAt?$AA?3?$AA?5?$AAT?$AA1?$AA_?$AAA?$AAB?$AAO?$AAR?$AAT?$AA_@ 10004638     smclib:smcprot.obj
 0001:00003690       ??_C@_1FC@EKCOEDDN@?$AA?$CF?$AAs?$AA?$CB?$AAS?$AAm?$AAa?$AAr?$AAt?$AAc?$AAa?$AAr?$AAd?$AAT?$AA1?$AAR?$AAe?$AAq?$AAu?$AAe?$AAs?$AAt?$AA?3?$AA?5?$AAT?$AA1?$AA_?$AAA?$AAB?$AAO?$AAR?$AAT?$AA_@ 10004690     smclib:smcprot.obj
 0001:000036e8       ??_C@_1FG@OKBNBILP@?$AA?$CF?$AAs?$AA?$CB?$AAS?$AAm?$AAa?$AAr?$AAt?$AAc?$AAa?$AAr?$AAd?$AAT?$AA1?$AAR?$AAe?$AAq?$AAu?$AAe?$AAs?$AAt?$AA?3?$AA?5?$AAT?$AA1?$AA_?$AAR?$AAE?$AAS?$AAY?$AAN?$AAC@ 100046e8     smclib:smcprot.obj
 0001:00003740       ??_C@_1FA@FDHCJOOF@?$AA?$CF?$AAs?$AA?$CB?$AAS?$AAm?$AAa?$AAr?$AAt?$AAc?$AAa?$AAr?$AAd?$AAT?$AA1?$AAR?$AAe?$AAq?$AAu?$AAe?$AAs?$AAt?$AA?3?$AA?5?$AAT?$AA1?$AA_?$AAI?$AAF?$AAS?$AA_?$AAR?$AAE@ 10004740     smclib:smcprot.obj
 0001:00003790       ??_C@_1EC@BFAGKBDF@?$AA?$CF?$AAs?$AA?$CB?$AAS?$AAm?$AAa?$AAr?$AAt?$AAc?$AAa?$AAr?$AAd?$AAT?$AA1?$AAR?$AAe?$AAq?$AAu?$AAe?$AAs?$AAt?$AA?3?$AA?5?$AAR?$AA?$CI?$AA?$CF?$AAd?$AA?$CJ?$AA?5?$AA?9?$AA?$DO?$AA?6@ 10004790     smclib:smcprot.obj
 0001:000037d8       ??_C@_1EI@EMIDDMNE@?$AA?$CF?$AAs?$AA?$CB?$AAS?$AAm?$AAa?$AAr?$AAt?$AAc?$AAa?$AAr?$AAd?$AAT?$AA1?$AAR?$AAe?$AAq?$AAu?$AAe?$AAs?$AAt?$AA?3?$AA?5?$AAI?$AA?$CI?$AA?$CF?$AAd?$AA?4?$AA?$CF?$AAd?$AA?$CJ?$AA?5@ 100047d8     smclib:smcprot.obj
 0001:00003820       ??_C@_1EO@MBAEMOOJ@?$AA?$CF?$AAs?$AA?$CB?$AAS?$AAm?$AAa?$AAr?$AAt?$AAc?$AAa?$AAr?$AAd?$AAT?$AA1?$AAR?$AAe?$AAq?$AAu?$AAe?$AAs?$AAt?$AA?3?$AA?5?$AAT?$AA1?$AA_?$AAI?$AAF?$AAS?$AA_?$AAR?$AAE@ 10004820     smclib:smcprot.obj
 0001:00003870       ??_C@_1FC@FBCCGBDK@?$AA?$CF?$AAs?$AA?$CB?$AAS?$AAm?$AAa?$AAr?$AAt?$AAc?$AAa?$AAr?$AAd?$AAT?$AA1?$AAR?$AAe?$AAq?$AAu?$AAe?$AAs?$AAt?$AA?3?$AA?5?$AAN?$AAA?$AAD?$AA?5?$AAs?$AAe?$AAt?$AA?5?$AAt@ 10004870     smclib:smcprot.obj
 0001:000038c4       ??_C@_1DM@BNJDCAJL@?$AA?$CF?$AAs?$AA?$CB?$AAS?$AAm?$AAa?$AAr?$AAt?$AAc?$AAa?$AAr?$AAd?$AAT?$AA1?$AAR?$AAe?$AAq?$AAu?$AAe?$AAs?$AAt?$AA?3?$AA?5?$AAT?$AA1?$AA_?$AA?$CF?$AAs?$AA?6?$AA?$AA@ 100048c4     smclib:smcprot.obj
 0001:00003900       ??_C@_1BA@ICKDJNIF@?$AAR?$AAE?$AAS?$AAT?$AAA?$AAR?$AAT?$AA?$AA@ 10004900     smclib:smcprot.obj
 0001:00003910       ??_C@_1M@JPCOGECE@?$AAS?$AAT?$AAA?$AAR?$AAT?$AA?$AA@ 10004910     smclib:smcprot.obj
 0001:00003920       ??_C@_1IG@GENLNLNP@?$AAD?$AA?3?$AA?2?$AAy?$AAa?$AAm?$AAa?$AAf?$AAp?$AA?9?$AA1?$AA?2?$AAp?$AAu?$AAb?$AAl?$AAi?$AAc?$AA?2?$AAC?$AAO?$AAM?$AAM?$AAO?$AAN?$AA?2?$AAo?$AAa?$AAk?$AA?2?$AAd?$AAr@ 10004920     smclib:smcprot.obj
 0001:000039a8       ??_C@_1BM@PCDHIBBH@?$AA?6?$AA?5?$AA?5?$AA?5?$AAL?$AAR?$AAC?$AA?3?$AA?5?$AA?$CF?$AA0?$AA2?$AAX?$AA?$AA@ 100049a8     smclib:smcprot.obj
 0001:000039c4       ??_C@_1CG@DGGCIJMK@?$AA?6?$AA?5?$AA?5?$AA?5?$AAC?$AAR?$AAC?$AA?3?$AA?5?$AA?$CF?$AA0?$AA2?$AAX?$AA?5?$AA?$CF?$AA0?$AA2?$AAX?$AA?$AA@ 100049c4     smclib:smcprot.obj
 0001:000039ec       ??_C@_15FFDNOHIK@?$AA?9?$AA?5?$AA?$AA@ 100049ec     smclib:smcprot.obj
 0001:000039f8       ??_C@_1GA@NGCEGHBG@?$AA?5?$AA?5?$AA?5?$AAN?$AAA?$AAD?$AA?3?$AA?5?$AA?$CF?$AA0?$AA2?$AAX?$AA?6?$AA?5?$AA?5?$AA?5?$AAP?$AAC?$AAB?$AA?3?$AA?5?$AA?$CF?$AA0?$AA2?$AAX?$AA?6?$AA?5?$AA?5?$AA?5?$AAL?$AAE?$AAN@ 100049f8     smclib:smcprot.obj
 0001:00003a58       ??_C@_1GG@PHJBGHML@?$AA?$CF?$AAs?$AA?$CB?$AAS?$AAm?$AAa?$AAr?$AAt?$AAc?$AAa?$AAr?$AAd?$AAT?$AA1?$AAR?$AAe?$AAp?$AAl?$AAy?$AA?3?$AA?5?$AAT?$AAo?$AAo?$AA?5?$AAm?$AAa?$AAn?$AAy?$AA?5?$AAe?$AAr@ 10004a58     smclib:smcprot.obj
 0001:00003ac0       ??_C@_1DO@HGHNMEEM@?$AAS?$AAm?$AAa?$AAr?$AAt?$AAc?$AAa?$AAr?$AAd?$AAT?$AA1?$AAR?$AAe?$AAp?$AAl?$AAy?$AA?3?$AA?5?$AAI?$AAn?$AAv?$AAa?$AAl?$AAi?$AAd?$AA?5?$AAP?$AAc?$AAb?$AA?5?$AA?$AA@ 10004ac0     smclib:smcprot.obj
 0001:00003b00       ??_C@_1EK@FOBIAJHG@?$AA?$CF?$AAs?$AA?$CB?$AAS?$AAm?$AAa?$AAr?$AAt?$AAc?$AAa?$AAr?$AAd?$AAT?$AA1?$AAR?$AAe?$AAp?$AAl?$AAy?$AA?3?$AA?5?$AA?5?$AA?5?$AAT?$AA1?$AA_?$AAV?$AAP?$AAP?$AA_?$AAE?$AAR@ 10004b00     smclib:smcprot.obj
 0001:00003b50       ??_C@_1EO@EBLBFGIF@?$AA?$CF?$AAs?$AA?$CB?$AAS?$AAm?$AAa?$AAr?$AAt?$AAc?$AAa?$AAr?$AAd?$AAT?$AA1?$AAR?$AAe?$AAp?$AAl?$AAy?$AA?3?$AA?5?$AA?5?$AA?5?$AAT?$AA1?$AA_?$AAW?$AAT?$AAX?$AA_?$AAR?$AAE@ 10004b50     smclib:smcprot.obj
 0001:00003ba0       ??_C@_1FC@MCEGLIIO@?$AA?$CF?$AAs?$AA?$CB?$AAS?$AAm?$AAa?$AAr?$AAt?$AAc?$AAa?$AAr?$AAd?$AAT?$AA1?$AAR?$AAe?$AAp?$AAl?$AAy?$AA?3?$AA?5?$AA?5?$AA?5?$AAT?$AA1?$AA_?$AAA?$AAB?$AAO?$AAR?$AAT?$AA_@ 10004ba0     smclib:smcprot.obj
 0001:00003bf8       ??_C@_1EO@KHHPMFIC@?$AA?$CF?$AAs?$AA?$CB?$AAS?$AAm?$AAa?$AAr?$AAt?$AAc?$AAa?$AAr?$AAd?$AAT?$AA1?$AAR?$AAe?$AAp?$AAl?$AAy?$AA?3?$AA?5?$AA?5?$AA?5?$AAT?$AA1?$AA_?$AAI?$AAF?$AAS?$AA_?$AAR?$AAE@ 10004bf8     smclib:smcprot.obj
 0001:00003c48       ??_C@_1FG@GFAANBII@?$AA?$CF?$AAs?$AA?$CB?$AAS?$AAm?$AAa?$AAr?$AAt?$AAc?$AAa?$AAr?$AAd?$AAT?$AA1?$AAR?$AAe?$AAp?$AAl?$AAy?$AA?3?$AA?5?$AA?5?$AA?5?$AAC?$AAa?$AAr?$AAd?$AA?5?$AAr?$AAe?$AAp?$AAo@ 10004c48     smclib:smcprot.obj
 0001:00003ca0       ??_C@_1EC@ODHNDHAL@?$AA?$CF?$AAs?$AA?$CB?$AAS?$AAm?$AAa?$AAr?$AAt?$AAc?$AAa?$AAr?$AAd?$AAT?$AA1?$AAR?$AAe?$AAp?$AAl?$AAy?$AA?3?$AA?5?$AA?5?$AA?5?$AAR?$AA?$CI?$AA?$CF?$AAd?$AA?$CJ?$AA?5?$AA?$DM?$AA?9?$AA?6@ 10004ca0     smclib:smcprot.obj
 0001:00003ce8       ??_C@_1FK@BKFOHPHP@?$AA?$CF?$AAs?$AA?$CB?$AAS?$AAm?$AAa?$AAr?$AAt?$AAc?$AAa?$AAr?$AAd?$AAT?$AA1?$AAR?$AAe?$AAp?$AAl?$AAy?$AA?3?$AA?5?$AAB?$AAl?$AAo?$AAc?$AAk?$AA?5?$AAn?$AAu?$AAm?$AAb?$AAe@ 10004ce8     smclib:smcprot.obj
 0001:00003d48       ??_C@_1EI@JEKKADNA@?$AA?$CF?$AAs?$AA?$CB?$AAS?$AAm?$AAa?$AAr?$AAt?$AAc?$AAa?$AAr?$AAd?$AAT?$AA1?$AAR?$AAe?$AAp?$AAl?$AAy?$AA?3?$AA?5?$AA?5?$AA?5?$AAI?$AA?$CI?$AA?$CF?$AAd?$AA?4?$AA?$CF?$AAd?$AA?$CJ?$AA?5@ 10004d48     smclib:smcprot.obj
 0001:00003d90       ??_C@_1FI@GCCNKNIM@?$AA?$CF?$AAs?$AA?$CB?$AAS?$AAm?$AAa?$AAr?$AAt?$AAc?$AAa?$AAr?$AAd?$AAT?$AA1?$AAR?$AAe?$AAp?$AAl?$AAy?$AA?3?$AA?5?$AA?5?$AA?5?$AAT?$AA1?$AA_?$AAR?$AAE?$AAS?$AAY?$AAN?$AAC@ 10004d90     smclib:smcprot.obj
 0001:00003de8       ??_C@_1IM@EDAGLLHL@?$AA?$CF?$AAs?$AA?$CB?$AAS?$AAm?$AAa?$AAr?$AAt?$AAc?$AAa?$AAr?$AAd?$AAT?$AA1?$AAR?$AAe?$AAp?$AAl?$AAy?$AA?3?$AA?5?$AA?5?$AA?5?$AAC?$AAa?$AAr?$AAd?$AA?5?$AAr?$AAe?$AAs?$AAp@ 10004de8     smclib:smcprot.obj
 0001:00003e78       ??_C@_1HE@MGIAIEPD@?$AA?$CF?$AAs?$AA?$CB?$AAS?$AAm?$AAa?$AAr?$AAt?$AAc?$AAa?$AAr?$AAd?$AAT?$AA1?$AAR?$AAe?$AAp?$AAl?$AAy?$AA?3?$AA?5?$AA?5?$AA?5?$AAC?$AAa?$AAr?$AAd?$AA?5?$AAd?$AAo?$AAe?$AAs@ 10004e78     smclib:smcprot.obj
 0001:00003ef0       ??_C@_1FA@ECKJJDHK@?$AA?$CF?$AAs?$AA?$CB?$AAS?$AAm?$AAa?$AAr?$AAt?$AAc?$AAa?$AAr?$AAd?$AAT?$AA1?$AAR?$AAe?$AAp?$AAl?$AAy?$AA?3?$AA?5?$AA?5?$AA?5?$AAT?$AA1?$AA_?$AAI?$AAF?$AAS?$AA_?$AAR?$AAE@ 10004ef0     smclib:smcprot.obj
 0001:00003f40       ??_C@_1EG@POCHCDGB@?$AA?$CF?$AAs?$AA?$CB?$AAS?$AAm?$AAa?$AAr?$AAt?$AAc?$AAa?$AAr?$AAd?$AAT?$AA1?$AAR?$AAe?$AAp?$AAl?$AAy?$AA?3?$AA?5?$AAB?$AAa?$AAd?$AA?5?$AAc?$AAh?$AAe?$AAc?$AAk?$AAs?$AAu@ 10004f40     smclib:smcprot.obj
 0001:00003f88       ??_C@_1FM@KMABPACM@?$AA?$CF?$AAs?$AA?$CB?$AAS?$AAm?$AAa?$AAr?$AAt?$AAc?$AAa?$AAr?$AAd?$AAT?$AA1?$AAR?$AAe?$AAp?$AAl?$AAy?$AA?3?$AA?5?$AAP?$AAa?$AAc?$AAk?$AAe?$AAt?$AA?5?$AAl?$AAe?$AAn?$AAg@ 10004f88     smclib:smcprot.obj
 0001:00003fe4       ??_C@_1BO@DHPPOOGN@?$AAG?$AAE?$AAT?$AA_?$AAL?$AAA?$AAS?$AAT?$AA_?$AAE?$AAR?$AAR?$AAO?$AAR?$AA?$AA@ 10004fe4     smclib:smcioctl.obj
 0001:00004004       ??_C@_1BE@DCOOAGKL@?$AAG?$AAE?$AAT?$AA_?$AAS?$AAT?$AAA?$AAT?$AAE?$AA?$AA@ 10005004     smclib:smcioctl.obj
 0001:00004018       ??_C@_1BK@IAGCDFCD@?$AAS?$AAE?$AAT?$AA_?$AAP?$AAR?$AAO?$AAT?$AAO?$AAC?$AAO?$AAL?$AA?$AA@ 10005018     smclib:smcioctl.obj
 0001:00004034       ??_C@_1BE@EHPIEKBH@?$AAI?$AAS?$AA_?$AAA?$AAB?$AAS?$AAE?$AAN?$AAT?$AA?$AA@ 10005034     smclib:smcioctl.obj
 0001:00004048       ??_C@_1BG@MPKKOEGO@?$AAI?$AAS?$AA_?$AAP?$AAR?$AAE?$AAS?$AAE?$AAN?$AAT?$AA?$AA@ 10005048     smclib:smcioctl.obj
 0001:00004060       ??_C@_1BA@EJLFONNA@?$AAS?$AAW?$AAA?$AAL?$AAL?$AAO?$AAW?$AA?$AA@ 10005060     smclib:smcioctl.obj
 0001:00004070       ??_C@_1M@JKMECKH@?$AAE?$AAJ?$AAE?$AAC?$AAT?$AA?$AA@ 10005070     smclib:smcioctl.obj
 0001:0000407c       ??_C@_1BC@MBPMHNIE@?$AAT?$AAR?$AAA?$AAN?$AAS?$AAM?$AAI?$AAT?$AA?$AA@ 1000507c     smclib:smcioctl.obj
 0001:00004090       ??_C@_1BG@DMKNPBCL@?$AAC?$AAO?$AAN?$AAF?$AAI?$AAS?$AAC?$AAA?$AAT?$AAE?$AA?$AA@ 10005090     smclib:smcioctl.obj
 0001:000040a8       ??_C@_1BM@IJDCIKJH@?$AAS?$AAE?$AAT?$AA_?$AAA?$AAT?$AAT?$AAR?$AAI?$AAB?$AAU?$AAT?$AAE?$AA?$AA@ 100050a8     smclib:smcioctl.obj
 0001:000040c4       ??_C@_1BM@JELKKPDD@?$AAG?$AAE?$AAT?$AA_?$AAA?$AAT?$AAT?$AAR?$AAI?$AAB?$AAU?$AAT?$AAE?$AA?$AA@ 100050c4     smclib:smcioctl.obj
 0001:000040e0       ??_C@_1M@LGJCJJJI@?$AAP?$AAO?$AAW?$AAE?$AAR?$AA?$AA@ 100050e0     smclib:smcioctl.obj
 0001:000040ec       ??_C@_1CA@HAEGBHBA@?$AA?$CK?$AA?$CK?$AA?$CK?$AA?5?$AAU?$AAN?$AAK?$AAN?$AAO?$AAW?$AAN?$AA?5?$AA?$CK?$AA?$CK?$AA?$CK?$AA?$AA@ 100050ec     smclib:smcioctl.obj
 0001:00004110       ??_C@_1II@JFCADGO@?$AAD?$AA?3?$AA?2?$AAy?$AAa?$AAm?$AAa?$AAf?$AAp?$AA?9?$AA1?$AA?2?$AAp?$AAu?$AAb?$AAl?$AAi?$AAc?$AA?2?$AAC?$AAO?$AAM?$AAM?$AAO?$AAN?$AA?2?$AAo?$AAa?$AAk?$AA?2?$AAd?$AAr@ 10005110     smclib:smcioctl.obj
 0001:000041b8       BSPGetSIMCLK               100051b8 f   bspsim.obj
 0001:00004228       BSPSetSIMClockGatingMode   10005228 f   bspsim.obj
 0001:0000432c       BSPSimIomuxSetPin          1000532c f   bspsim.obj
 0001:0000461c       BSPSimSelect3Volts         1000561c f   bspsim.obj
 0001:00004630       DllEntry                   10005630 f   sim_common_topaz_v1:simce.obj
 0001:0000472c       SCR_Init                   1000572c f   sim_common_topaz_v1:simce.obj
 0001:00004930       SCR_Deinit                 10005930 f   sim_common_topaz_v1:simce.obj
 0001:000049c4       SCR_Open                   100059c4 f   sim_common_topaz_v1:simce.obj
 0001:00004f44       SCR_Close                  10005f44 f   sim_common_topaz_v1:simce.obj
 0001:000051e4       SCR_IOControl              100061e4 f   sim_common_topaz_v1:simce.obj
 0001:000053f0       SCR_Read                   100063f0 f   sim_common_topaz_v1:simce.obj
 0001:00005418       SCR_Write                  10006418 f   sim_common_topaz_v1:simce.obj
 0001:00005440       SCR_Seek                   10006440 f   sim_common_topaz_v1:simce.obj
 0001:00005468       SCR_PowerUp                10006468 f   sim_common_topaz_v1:simce.obj
 0001:000054b0       SCR_PowerDown              100064b0 f   sim_common_topaz_v1:simce.obj
 0001:0000623c       CBCardPower                1000723c f   sim_common_topaz_v1:simcb.obj
 0001:000064e4       CBSetProtocol              100074e4 f   sim_common_topaz_v1:simcb.obj
 0001:00006934       CBTransmit                 10007934 f   sim_common_topaz_v1:simcb.obj
 0001:00006fc0       CBCardTracking             10007fc0 f   sim_common_topaz_v1:simcb.obj
 0001:00007248       CBUpdateCardState          10008248 f   sim_common_topaz_v1:simcb.obj
 0001:00007348       SIM_InternalMapRegisterAddresses 10008348 f   sim_common_topaz_v1:simhw.obj
 0001:00007440       SIM_InternalUnMapRegisterAddresses 10008440 f   sim_common_topaz_v1:simhw.obj
 0001:000074e0       SIM_Init                   100084e0 f   sim_common_topaz_v1:simhw.obj
 0001:00007954       SIM_Open                   10008954 f   sim_common_topaz_v1:simhw.obj
 0001:00007a74       SIM_Close                  10008a74 f   sim_common_topaz_v1:simhw.obj
 0001:00007c50       SIM_ColdReset              10008c50 f   sim_common_topaz_v1:simhw.obj
 0001:00008a4c       SIM_WarmReset              10009a4c f   sim_common_topaz_v1:simhw.obj
 0001:00008e34       SIM_ReadData               10009e34 f   sim_common_topaz_v1:simhw.obj
 0001:0000922c       SIM_WriteData              1000a22c f   sim_common_topaz_v1:simhw.obj
 0001:00009468       SIM_Deactivate             1000a468 f   sim_common_topaz_v1:simhw.obj
 0001:00009630       SIM_ConfigCLK              1000a630 f   sim_common_topaz_v1:simhw.obj
 0001:00009bd0       SIM_ConfigTime             1000abd0 f   sim_common_topaz_v1:simhw.obj
 0001:00009cd0       SIM_CheckCard              1000acd0 f   sim_common_topaz_v1:simhw.obj
 0001:0000a078       SIM_FlushFIFO              1000b078 f   sim_common_topaz_v1:simhw.obj
 0001:0000a194       Dump_Registers             1000b194 f   sim_common_topaz_v1:simhw.obj
 0001:0000a3b4       ResetEvent                 1000b3b4 f i sim_common_topaz_v1:simhw.obj
 0001:0000a3ec       DeleteCriticalSection      1000b3ec f   coredll:COREDLL.dll
 0001:0000a3fc       DisableThreadLibraryCalls  1000b3fc f   coredll:COREDLL.dll
 0001:0000a40c       InitializeCriticalSection  1000b40c f   coredll:COREDLL.dll
 0001:0000a41c       NKDbgPrintfW               1000b41c f   coredll:COREDLL.dll
 0001:0000a42c       RegisterDbgZones           1000b42c f   coredll:COREDLL.dll
 0001:0000a43c       LeaveCriticalSection       1000b43c f   coredll:COREDLL.dll
 0001:0000a44c       EnterCriticalSection       1000b44c f   coredll:COREDLL.dll
 0001:0000a45c       InterlockedDecrement       1000b45c f   coredll:COREDLL.dll
 0001:0000a46c       Sleep                      1000b46c f   coredll:COREDLL.dll
 0001:0000a47c       CreateThread               1000b47c f   coredll:COREDLL.dll
 0001:0000a48c       SetLastError               1000b48c f   coredll:COREDLL.dll
 0001:0000a49c       InterlockedIncrement       1000b49c f   coredll:COREDLL.dll
 0001:0000a4ac       CloseHandle                1000b4ac f   coredll:COREDLL.dll
 0001:0000a4bc       WaitForSingleObject        1000b4bc f   coredll:COREDLL.dll
 0001:0000a4cc       StringCchCopyW             1000b4cc f   coredll:COREDLL.dll
 0001:0000a4dc       LocalAlloc                 1000b4dc f   coredll:COREDLL.dll
 0001:0000a4ec       RegCloseKey                1000b4ec f   coredll:COREDLL.dll
 0001:0000a4fc       RegQueryValueExW           1000b4fc f   coredll:COREDLL.dll
 0001:0000a50c       OpenDeviceKey              1000b50c f   coredll:COREDLL.dll
 0001:0000a51c       RegOpenKeyExW              1000b51c f   coredll:COREDLL.dll
 0001:0000a52c       StringCchCatW              1000b52c f   coredll:COREDLL.dll
 0001:0000a53c       LocalFree                  1000b53c f   coredll:COREDLL.dll
 0001:0000a54c       InterruptInitialize        1000b54c f   coredll:COREDLL.dll
 0001:0000a55c       KernelIoControl            1000b55c f   coredll:COREDLL.dll
 0001:0000a56c       CreateEventW               1000b56c f   coredll:COREDLL.dll
 0001:0000a57c       InterruptDisable           1000b57c f   coredll:COREDLL.dll
 0001:0000a58c       InterruptDone              1000b58c f   coredll:COREDLL.dll
 0001:0000a59c       EventModify                1000b59c f   coredll:COREDLL.dll
 0001:0000a5ac       MmMapIoSpace               1000b5ac f   ceddk:CEDDK.dll
 0001:0000a5bc       MmUnmapIoSpace             1000b5bc f   ceddk:CEDDK.dll
 0001:0000a5cc       DDKClockGetFreq            1000b5cc f   cspddk:CSPDDK.dll
 0001:0000a5dc       DDKClockSetGatingMode      1000b5dc f   cspddk:CSPDDK.dll
 0001:0000a5ec       DDKGpioWriteDataPin        1000b5ec f   cspddk:CSPDDK.dll
 0001:0000a5fc       DDKGpioSetConfig           1000b5fc f   cspddk:CSPDDK.dll
 0001:0000a60c       DDKIomuxSetPadConfig       1000b60c f   cspddk:CSPDDK.dll
 0001:0000a61c       DDKIomuxSetPinMux          1000b61c f   cspddk:CSPDDK.dll
 0001:0000a62c       SmartcardCreateLink        1000b62c f   smclib:smcce.obj
 0001:0000a768       SmartcardDeleteLink        1000b768 f   smclib:smcce.obj
 0001:0000a820       SmartcardInitialize        1000b820 f   smclib:smcce.obj
 0001:0000acdc       SmartcardExit              1000bcdc f   smclib:smcce.obj
 0001:0000af44       SmartcardDeviceControl     1000bf44 f   smclib:smcce.obj
 0001:0000b7a4       SmartcardCompleteCardTracking 1000c7a4 f   smclib:smcce.obj
 0001:0000b7d0       MapNtStatusToWinError      1000c7d0 f   smclib:smcce.obj
 0001:0000b8e0       SetEvent                   1000c8e0 f i smclib:smcce.obj
 0001:0000b918       SmartcardGetDebugLevel     1000c918 f   smclib:smcutil.obj
 0001:0000b938       SmartcardSetDebugLevel     1000c938 f   smclib:smcutil.obj
 0001:0000b95c       DumpData                   1000c95c f   smclib:smcutil.obj
 0001:0000ba80       SmartcardInitializeCardCapabilities 1000ca80 f   smclib:smcutil.obj
 0001:0000bbe4       SmartcardInvertData        1000cbe4 f   smclib:smcutil.obj
 0001:0000bcd0       SmartcardUpdateCardCapabilities 1000ccd0 f   smclib:smcutil.obj
 0001:0000d768       SmartcardRawRequest        1000e768 f   smclib:smcprot.obj
 0001:0000d91c       SmartcardRawReply          1000e91c f   smclib:smcprot.obj
 0001:0000d9b4       SmartcardT0Request         1000e9b4 f   smclib:smcprot.obj
 0001:0000dcf8       SmartcardT0Reply           1000ecf8 f   smclib:smcprot.obj
 0001:0000de58       SmartcardT1Chksum          1000ee58 f   smclib:smcprot.obj
 0001:0000e26c       SmartcardT1Request         1000f26c f   smclib:smcprot.obj
 0001:0000f148       SmartcardT1Reply           10010148 f   smclib:smcprot.obj
 0001:000100c0       ULongAdd                   100110c0 f i smclib:smcprot.obj
 0001:00010134       CeULongAdd3                10011134 f i smclib:smcprot.obj
 0001:000101b0       MapIoControlCodeToString   100111b0 f   smclib:smcioctl.obj
 0001:00010250       SMCDeviceIoControl         10011250 f   smclib:smcioctl.obj
 0001:00011e94       __security_init_cookie     10012e94 f   corelib0:seccinit.obj
 0001:00011f5c       __GSHandlerCheck           10012f5c f   corelib0:gshandler.obj
 0001:00011fa4       __GSHandlerCheckCommon     10012fa4 f   corelib0:gshandler.obj
 0001:0001204c       __security_check_cookie    1001304c f   corelib0:armsecgs.obj
 0001:00012060       __gsfailure                10013060 f   corelib0:armsecgs.obj
 0001:000120a4       memset                     100130a4 f   corelib1:COREDLL.dll
 0001:000120b4       memcpy                     100130b4 f   corelib1:COREDLL.dll
 0001:000120c4       wcslen                     100130c4 f   corelib1:COREDLL.dll
 0001:000120d4       mbstowcs                   100130d4 f   corelib1:COREDLL.dll
 0001:000120e4       __rt_udiv                  100130e4 f   corelib1:COREDLL.dll
 0001:000120f4       memcmp                     100130f4 f   corelib1:COREDLL.dll
 0001:00012104       __rt_sdiv                  10013104 f   corelib1:COREDLL.dll
 0001:00012114       __C_specific_handler       10013114 f   corelib1:COREDLL.dll
 0001:00012124       __security_gen_cookie2     10013124 f   corelib1:COREDLL.dll
 0001:00012134       __report_gsfailure         10013134 f   corelib1:COREDLL.dll
 0001:00012144       CspSIMGetIRQs              10013144 f   sim_mx25_topaz_v1:cspsim.obj
 0001:00012234       CspSIMGetBaseAddress       10013234 f   sim_mx25_topaz_v1:cspsim.obj
 0001:000122a0       GetProcAddressW            100132a0 f   coredll:COREDLL.dll
 0001:000122b0       GetModuleHandleW           100132b0 f   coredll:COREDLL.dll
 0001:000122c0       CloseMsgQueue              100132c0 f   coredll:COREDLL.dll
 0001:000122d0       StopPowerNotifications     100132d0 f   coredll:COREDLL.dll
 0001:000122e0       ReadMsgQueue               100132e0 f   coredll:COREDLL.dll
 0001:000122f0       WaitForMultipleObjects     100132f0 f   coredll:COREDLL.dll
 0001:00012300       RequestPowerNotifications  10013300 f   coredll:COREDLL.dll
 0001:00012310       CreateMsgQueue             10013310 f   coredll:COREDLL.dll
 0001:00012320       OutputDebugStringW         10013320 f   coredll:COREDLL.dll
 0001:00012370       __IMPORT_DESCRIPTOR_COREDLL 10013370     coredll:COREDLL.dll
 0001:00012384       __IMPORT_DESCRIPTOR_CEDDK  10013384     ceddk:CEDDK.dll
 0001:00012398       __IMPORT_DESCRIPTOR_CSPDDK 10013398     cspddk:CSPDDK.dll
 0001:000123ac       __NULL_IMPORT_DESCRIPTOR   100133ac     coredll:COREDLL.dll
 0002:00000000       __imp_MmMapIoSpace         10014000     ceddk:CEDDK.dll
 0002:00000004       __imp_MmUnmapIoSpace       10014004     ceddk:CEDDK.dll
 0002:00000008       \177CEDDK_NULL_THUNK_DATA  10014008     ceddk:CEDDK.dll
 0002:0000000c       __imp_NKDbgPrintfW         1001400c     coredll:COREDLL.dll
 0002:00000010       __imp_RegisterDbgZones     10014010     coredll:COREDLL.dll
 0002:00000014       __imp_LeaveCriticalSection 10014014     coredll:COREDLL.dll
 0002:00000018       __imp_EnterCriticalSection 10014018     coredll:COREDLL.dll
 0002:0000001c       __imp_InterlockedDecrement 1001401c     coredll:COREDLL.dll
 0002:00000020       __imp_Sleep                10014020     coredll:COREDLL.dll
 0002:00000024       __imp_CreateThread         10014024     coredll:COREDLL.dll
 0002:00000028       __imp_SetLastError         10014028     coredll:COREDLL.dll
 0002:0000002c       __imp_InterlockedIncrement 1001402c     coredll:COREDLL.dll
 0002:00000030       __imp_CloseHandle          10014030     coredll:COREDLL.dll
 0002:00000034       __imp_WaitForSingleObject  10014034     coredll:COREDLL.dll
 0002:00000038       __imp_StringCchCopyW       10014038     coredll:COREDLL.dll
 0002:0000003c       __imp_LocalAlloc           1001403c     coredll:COREDLL.dll
 0002:00000040       __imp_InitializeCriticalSection 10014040     coredll:COREDLL.dll
 0002:00000044       __imp_RegQueryValueExW     10014044     coredll:COREDLL.dll
 0002:00000048       __imp_OpenDeviceKey        10014048     coredll:COREDLL.dll
 0002:0000004c       __imp_RegOpenKeyExW        1001404c     coredll:COREDLL.dll
 0002:00000050       __imp_StringCchCatW        10014050     coredll:COREDLL.dll
 0002:00000054       __imp_LocalFree            10014054     coredll:COREDLL.dll
 0002:00000058       __imp_InterruptInitialize  10014058     coredll:COREDLL.dll
 0002:0000005c       __imp_KernelIoControl      1001405c     coredll:COREDLL.dll
 0002:00000060       __imp_CreateEventW         10014060     coredll:COREDLL.dll
 0002:00000064       __imp_InterruptDisable     10014064     coredll:COREDLL.dll
 0002:00000068       __imp_InterruptDone        10014068     coredll:COREDLL.dll
 0002:0000006c       __imp_EventModify          1001406c     coredll:COREDLL.dll
 0002:00000070       __imp_DeleteCriticalSection 10014070     coredll:COREDLL.dll
 0002:00000074       __imp_DisableThreadLibraryCalls 10014074     coredll:COREDLL.dll
 0002:00000078       __imp_RegCloseKey          10014078     coredll:COREDLL.dll
 0002:0000007c       __imp_CreateMsgQueue       1001407c     coredll:COREDLL.dll
 0002:00000080       __imp_RequestPowerNotifications 10014080     coredll:COREDLL.dll
 0002:00000084       __imp_WaitForMultipleObjects 10014084     coredll:COREDLL.dll
 0002:00000088       __imp_ReadMsgQueue         10014088     coredll:COREDLL.dll
 0002:0000008c       __imp_StopPowerNotifications 1001408c     coredll:COREDLL.dll
 0002:00000090       __imp_CloseMsgQueue        10014090     coredll:COREDLL.dll
 0002:00000094       __imp_GetModuleHandleW     10014094     coredll:COREDLL.dll
 0002:00000098       __imp_memset               10014098     corelib1:COREDLL.dll
 0002:0000009c       __imp_memcpy               1001409c     corelib1:COREDLL.dll
 0002:000000a0       __imp_wcslen               100140a0     corelib1:COREDLL.dll
 0002:000000a4       __imp_mbstowcs             100140a4     corelib1:COREDLL.dll
 0002:000000a8       __imp___rt_udiv            100140a8     corelib1:COREDLL.dll
 0002:000000ac       __imp_memcmp               100140ac     corelib1:COREDLL.dll
 0002:000000b0       __imp___rt_sdiv            100140b0     corelib1:COREDLL.dll
 0002:000000b4       __imp___C_specific_handler 100140b4     corelib1:COREDLL.dll
 0002:000000b8       __imp___security_gen_cookie2 100140b8     corelib1:COREDLL.dll
 0002:000000bc       __imp___report_gsfailure   100140bc     corelib1:COREDLL.dll
 0002:000000c0       __imp_GetProcAddressW      100140c0     coredll:COREDLL.dll
 0002:000000c4       __imp_OutputDebugStringW   100140c4     coredll:COREDLL.dll
 0002:000000c8       \177COREDLL_NULL_THUNK_DATA 100140c8     coredll:COREDLL.dll
 0002:000000cc       __imp_DDKIomuxSetPadConfig 100140cc     cspddk:CSPDDK.dll
 0002:000000d0       __imp_DDKGpioSetConfig     100140d0     cspddk:CSPDDK.dll
 0002:000000d4       __imp_DDKGpioWriteDataPin  100140d4     cspddk:CSPDDK.dll
 0002:000000d8       __imp_DDKClockSetGatingMode 100140d8     cspddk:CSPDDK.dll
 0002:000000dc       __imp_DDKClockGetFreq      100140dc     cspddk:CSPDDK.dll
 0002:000000e0       __imp_DDKIomuxSetPinMux    100140e0     cspddk:CSPDDK.dll
 0002:000000e4       \177CSPDDK_NULL_THUNK_DATA 100140e4     cspddk:CSPDDK.dll
 0002:000000e8       dpCurSettings              100140e8     sim_common_topaz_v1:simce.obj
 0002:000008b8       __security_cookie          100148b8     corelib0:seccinit.obj
 0002:000008bc       __security_cookie_complement 100148bc     corelib0:seccinit.obj
 0002:000008c4       g_pfnIntroduceReader       100148c4     smclib:smcce.obj
 0002:000008c8       g_pfnForgetReader          100148c8     smclib:smcce.obj
 0002:000008e0       g_DriverCritSect           100148e0     <common>
 0002:000008f8       g_DeviceSlot               100148f8     <common>
 0002:00000900       DebugLevel                 10014900     <common>
 0002:00000904       g_hReEnumerationEvent      10014904     <common>
 0002:00000908       g_IsResumed                10014908     <common>

 entry point at        0001:00004630

 Static symbols

 0001:00004868       AddDevice                  10005868 f   sim_common_topaz_v1:simce.obj
 0001:00004c70       ValidateAndEnterDevice     10005c70 f   sim_common_topaz_v1:simce.obj
 0001:00004d78       SIMCardDetectionThread     10005d78 f   sim_common_topaz_v1:simce.obj
 0001:00005500       SIMLoadDevice              10006500 f   sim_common_topaz_v1:simce.obj
 0001:00005a34       SIMVendorIoctl             10006a34 f   sim_common_topaz_v1:simce.obj
 0001:00005b60       GetIOIndex                 10006b60 f   sim_common_topaz_v1:simce.obj
 0001:00005d38       GetDeviceName              10006d38 f   sim_common_topaz_v1:simce.obj
 0001:00005e6c       MakeFriendlyName           10006e6c f   sim_common_topaz_v1:simce.obj
 0001:00005f20       SIMUnloadDevice            10006f20 f   sim_common_topaz_v1:simce.obj
 0001:00006168       RemoveDevice               10007168 f   sim_common_topaz_v1:simce.obj
 0001:00006aa4       CBT0Transmit               10007aa4 f   sim_common_topaz_v1:simcb.obj
 0001:00006bd8       T0_ExchangeData            10007bd8 f   sim_common_topaz_v1:simcb.obj
 0001:00007068       CBSynchronizeSIM           10008068 f   sim_common_topaz_v1:simcb.obj
 0001:00009db8       SIM_MaskInterrupts         1000adb8 f   sim_common_topaz_v1:simhw.obj
 0001:0000d708       Pow2                       1000e708 f   smclib:smcutil.obj
 0001:0000d868       IsRoomForRequest           1000e868 f   smclib:smcprot.obj
 0001:0000ef7c       DumpT1Block                1000ff7c f   smclib:smcprot.obj
